:106DEE000000770200000301FA0400EF0500030A19
:106DFE000A5A0B001E0C00FA0D00030E00040F01C0
:106E0E0064100096120132130AFA14010217010AD5
:106E1E001801EF1905321A010A1B01EF1C05321F6A
:106E2E00FFFF20FFFF23011E2400642A00FA2B001F
:106E3E00FA2C50782D003C2E0046300064325078EB
:106E4E003300003432FF35016436016437015038A7
:106E5E000A643A00033B00043C00643E003C3F00E1
:106E6E000040FFFF411450420A5A430AC8440532FB
:106E7E004500B44600FA4900024B00014C00FA509E
:106E8E000606510596520A32530B46540A9657057A
:106E9E0046590A465A32FA5B010A5C0A325E000A09
:106EAE005F00646200FE64FFFF67FFFF6801016917
:106EBE0001016A05966B00006C32FF6D00047300D1
:106ECE00017400017801327901327E006481006420
:106EDE0084FFFF8800028A00019D0A969E00019F92
:106EEE00FFFFA0FFFFA2000AA3FFFFA40064A500FE
:106EFE0064A6FFFFA7FFFFA8FFFFA9FFFF01010385
:106F0E001501022F003C4701064802045601034EAC
:106F1E00FFFF58000261FFFF6600028500AF86008A
:106F2E00018700FA890109990006A100FAFAFAFA16
:106F3E000101031501022F1E3C47010648020456AB
:106F4E0001034EFFFF58000261FFFF66000285003D
:106F5E00AF8600018700FA890109990000A100009F
:106F6E00FAFAFA0101031501022F1E3C47010348EC
:106F7E0002035601014EFFFF58000061FFFF66003D
:106F8E000085FFFF86FFFF87FFFF89010299000042
:106F9E00A10000FAFAFA0065006F00790083008DF7
:106FAE00009700A100AC00B600C000CA00D400DEFD
:106FBE0000E800F200580060006800700078008061
:106FCE0000880090009800A000A800B000B800C192
:106FDE0000C800D000D800DF00E600EE00F6004149
:106FEE000047004D00530059005F0065006C0071B2
:106FFE000077007D00830089008F0095009B00A222
:10700E0000A700AC00B200B900C000C500CA00D293
:0A701E0000D500DD00E100E700EFFF
:103D750075A71085F97385FA747E017F00E57412C5
:103D8500713AE5732FFF50010E8E598F5A90001826
:103D9500E0FCA3E0FDEF2DFDEE3CFC8C5B8D5C9023
:103DA5000038E0FAA3E0FBED2BFBEC3AFA8A5B8BDB
:103DB5005C2275A71085F97385FA747E017F00E58D
:103DC5007412713AE5732FFF50010E8E598F5AAC5C
:103DD5002CAD2DEF2DFDEE3CFC8C5B8D5C90003801
:103DE500E0FAA3E0FBED2BFBEC3AFA8A5B8B5C2255
:103DF500E55CF5FBE55BF5FCD29322E55CF5E9E5D1
:103E05005BF5EAD29422E55CF5EBE55BF5ECD29146
:103E150022E55CF5EDE55BF5EED29222E55CF5FD7C
:103E2500E55BF5FED28722E55CF5CEE55BF5CFD205
:103E35009022A202B34008E5B54480F5B58006E5B9
:103E4500B5547FF5B522E50C906980F828287302F2
:103E55003EE7A233B34008E5B54408F5B58006E56D
:103E6500B554F7F5B5807BA233B34008E5B54402F8
:103E7500F5B58006E5B554FDF5B58066A233B340CA
:103E850008E5B54410F5B58006E5B554EFF5B58000
:103E950051A233B34008E5B54420F5B58006E5B534
:103EA50054DFF5B5803CA233B34008E5B54440F591
:103EB500B58006E5B554BFF5B58027A233B34008F4
:103EC500E5B54480F5B58006E5B5547FF5B58012B6
:103ED500A2339292800CA23392878006A2339290ED
:023EE50080005B
:10698000023E54023E57023E6C023E81023E960297
:106990003EAB023EC0023ED5023EDB023EE1023E7D
:0169A000E70F
:103EE70022744D900157F07469900158F0747490E2
:103EF7000159F0747390015AF0747590015BF07476
:103F07006290015CF0746990015DF0747390015EDA
:103F1700F0746890015FF07469900160F07420900C
:103F27000161F07436900162F07443900163F0749C
:103F370079900164F0746C900165F02290088EE02E
:103F4700FEA3E0FF741DD39F74019E400C906DEE9D
:103F5700120048E493F599804C90F802E493B40575
:103F67001490088EE0FEA3E0FF906E21120048E453
:103F770093F599803090F802E493D3940540149018
:103F8700088EE0FEA3E0FF906DEE120048E493F583
:103F970099801290088EE0FEA3E0FF906E54120005
:103FA70048E493F59990088E12714890088EE0FEC8
:103FB700A3E0FFEFB45007EEB40103754D0022AE46
:103FC70059AF5A74788E048F05FF12712A8C5B8D56
:103FD7005CAE59AF5A74788E048F05FF1271558CF9
:103FE700598D5AE55A455960137478C3955AFFE4B9
:103FF7009559FE8E598F5A785B12718DE573A85BC0
:10400700B80015D3955C4010E573C3955CFFE49544
:104017005BFE8E5B8F5C8010E5732403C3955CFFAA
:10402700E4955BFE8E5B8F5C22900094E0B4010404
:10403700C2088002D208900095E0B40104C209804A
:1040470002D2099000D2E075F0D7A4FFAEF0740A4F
:104057008E048F05FF12712A900882ECF0A3EDF011
:104067009000D2E075F02BA4FFAEF0900014EEF0B4
:10407700A3EFF07E017F00900090E012713A90006C
:10408700D3E08E048F05FF12712A740AFF12712A7A
:104097008D609000DCE075F0D7A4FFAEF0740A8E57
:1040A700048F05FF12712A900886ECF0A3EDF090BB
:1040B70000DEE060139000DEE0F5F0741684FF7E0A
:1040C70000EF9008E4F0800674649008E4F0900034
:1040D700D4E090006DF0900120E090007AF090011C
:1040E70022E0FE9000D0E08E0088F0A4FFAEF0EF53
:1040F7009008EDF09000FBE075F013A4FDACF09094
:104107000038ECF0A3EDF0A220B3401690016CE06C
:10411700700C90016DE0700690016EE06002800205
:10412700C22090016CE0B4300F90016DE0B44708F5
:1041370090016EE0643B60028004D2218002C221BC
:1041470090008DE0FE9008EEE06E601A7599E61219
:10415700019C74AB900047F01206DA750964750884
:104167000012062480FE900085E07006740090001F
:10417700BAF0900071E0FE9000BAE0B506639000D7
:1041870074E0FE9000D8E0B50657900072E0FE900C
:1041970000E6E0B5064B900078E0FE90008DE0B5B4
:1041A700063F900075E0FE9000C8E0B5063390002A
:1041B70073E0FE9000D6E0B50627900076E0FE900B
:1041C70000F3E0B5061B900077E0FE9000F4E0B541
:1041D700060F900079E0FE900106E06E700302443E
:1041E70090900095E070089000D6E064046002802B
:1041F7000674039000D6F090004FE0C39405500872
:104207007402900109F0801D9000C8E0D394025019
:10421700069000E6E060087406900109F0800674D5
:1042270009900109F090008DE0B401067400900038
:104237008DF090008DE0B4020674009000D8F090E5
:10424700008DE0B4030674009000E5F09000D8E01C
:10425700D394014026741B90010BF074009000A1C9
:10426700F074009006D6F074009006D7F09000BA6C
:10427700E0600674009000BAF080329000BAE06007
:104287001A740090010BF0741B9000A1F074009059
:1042970006D6F074009006D7F08012740090010BD8
:1042A700F074009000A1F0741B9006D6F09000C83F
:1042B700E0D3940240089000E6E0640260028006C2
:1042C70074009000E6F09000C8E0D3940240089094
:1042D70000E6E0640160028027741C90010CF07412
:1042E700009000A2F074009006DAF074009006DBEC
:1042F700F09000BAE0B4020674019000BAF080337F
:104307009000BAE0B4021A740090010CF0741C908B
:1043170000A2F074009006DAF074009006DBF080DB
:1043270012740090010CF074009000A2F0741C90BD
:1043370006DAF09000F3E06014740790010DF07452
:10434700009006CEF074009006CFF0800C740090B9
:10435700010DF074079006CEF09000F4E06014743D
:104367000890010EF074009006D2F074009006D306
:10437700F0800C740090010EF074089006D2F09053
:104387000106E06014742A90077EF074009006CA54
:10439700F074009006CBF0800C740090077EF074E8
:1043A7002A9006CAF09000C8E0B402069000E6E042
:1043B7006002802674049006DEF074059006E2F031
:1043C70074069006E6F07400900779F07400900781
:1043D7007AF0740090077BF0803674009006DEF068
:1043E70074009006DFF074009006E2F07400900607
:1043F700E3F074009006E6F074009006E7F07404AA
:10440700900779F0740590077AF0740690077BF0AF
:104417009000D6E0D3940240147418900771F0749A
:1044270019900772F0741A900773F0801274009055
:104437000771F07400900772F07400900773F0D260
:104447001F9000BAE0900071F09000E6E0900072D3
:10445700F09000D8E0900074F09000C8E0900075EC
:10446700F09000D6E0900073F090008DE090007817
:10447700F09000F3E0900076F09000F4E090007781
:10448700F0900106E0900079F09000F0E0B4011799
:10449700900024740FF0A374FFF0900026E4F0A3BB
:1044A700F074029000F0F09000F0E0B40341900047
:1044B70026E0FEA3E0FF900024E0FCA3E0FD1271DC
:1044C70085741012713A7408120039EF9000EFF0FA
:1044D700EF700674FF9000EFF074009000F0F0901A
:1044E7000025E09000A6F0900024E09000A7F0904F
:1044F7000081E090007EF0900080E090007DF090D9
:1045070000AFE0C3941E50569000AFE0F404241EA1
:1045170090007FF090007FE075F07884FF7E008F39
:104527007390007FE075F07884ADF07C008D749017
:10453700007DE0D39574400D90007DE0C3957490A5
:10454700007DF0800F90007DE02478C39574900083
:104557007DF0057390007EE0257390007EF090005B
:104567007EE0900040F0900040E004900041F09021
:104577000040E02402900042F0900040E0D3940312
:10458700400B900040E0C39403900040F09000413E
:10459700E0D39403400B900041E0C39403900041A3
:1045A700F0900042E0D39403400B900042E0C394A4
:1045B70003900042F0755D01900081E0FE9000C716
:1045C700E0D39E5013900081E0FE9000C7E0F40412
:1045D7002E04900043F08013900081E02406FE90A3
:1045E70000C7E0F4042E04900043F0900043E0D3AA
:1045F7009403400F900043E0C39403900043F0D22C
:104607001A8002C21A900043E004900044F0900020
:1046170043E02402900045F0900044E0D394034027
:104627000B900044E0C39403900044F0900045E0F1
:10463700D39403400B900045E0C39403900045F0EA
:1046470012019C22C293C294C291C292C287C290A5
:10465700E5B554EFF5B5E5B554DFF5B5C296C295A6
:10466700C2A0C297C2A2C2A1E5B554BFF5B5E5B5D0
:10467700547FF5B5E5B554FBF5B5C20A755E4690AE
:1046870000CAE07005756D028003756D03755400EF
:1046970075530090000C74FFF0A374DCF0C210C2D5
:1046A70012C21474C890003AF074C890003CF074B9
:1046B700C890003EF0755200755100C20375460060
:1046C700E56FB41303756F0075630090001AE4F08B
:1046D700A3F0757010C20DC20EC20FC2027556004C
:1046E70075550090000EE4F0A3F0900010E4F0A3DD
:1046F700F0C22375580075570090008CE075F032B2
:10470700A4FFAEF0900022EEF0A3EFF090007BE460
:10471700F09008EAE4F090007CE4F0C219C21AC2F3
:104727001B900012E4F0A3F0C204C20522755A00E0
:10473700755900AE59AF5A741CC39F74019E50033C
:10474700024828906DEE120048E493645F6023905E
:104757006DEE120048E493647E6017906DEE1200D0
:1047670048E4936481600B906DEE120048E493B4C3
:104777008403024808AE59AF5A906DEE120048E420
:104787009390008012716B0FBF00010EE0FC906DDB
:10479700EE120048ECFEE493FFEEC39F5026AE599D
:1047A700AF5A0FBF00010E906DEE120048AE59AF21
:1047B7005AE493FC906DEE120048E4939000801247
:1047C700716BECF0AE59AF5A906DEE120048E4935E
:1047D70090008012716BE0FC906DF0120048ECFCC9
:1047E700E493FDECD39D4019906DF0120048E493DB
:1047F700FC906DEE120048E49390008012716BEC10
:10480700F0AE59AF5A74022FFF50010E8E598F5ACE
:10481700785A740126F6500418E436F64003024726
:104827003A22755A00755900AE59AF5A7432BE0014
:10483700039F50030248F6906F0B120048E49390D1
:10484700008012716B0FBF00010EE0FC906F0B121E
:104857000048ECFEE493FFEEC39F5026AE59AF5AD3
:104867000FBF00010E906F0B120048AE59AF5AE40C
:1048770093FC906F0B120048E49390008012716BC9
:10488700ECF0AE59AF5A906F0B120048E4939000CA
:104897008012716BE0FC906F0D120048ECFCE49302
:1048A700FDECD39D4019906F0D120048E493FC90E6
:1048B7006F0B120048E49390008012716BECF0AE1E
:1048C70059AF5A742D6F4E7006755A33755900AE2D
:1048D70059AF5A74022FFF50010E8E598F5A785ACA
:1048E700740126F6500418E436F6400302482F22D6
:1048F700755A00755900AE59AF5A7432BE00039FFE
:1049070050030249C4906F3E120048E49390008020
:1049170012716B0FBF00010EE0FC906F3E12004852
:10492700ECFEE493FFEEC39F5026AE59AF5A0FBF7C
:1049370000010E906F3E120048AE59AF5AE493FC47
:10494700906F3E120048E49390008012716BECF078
:10495700AE59AF5A906F3E120048E4939000801210
:10496700716BE0FC906F40120048ECFCE493FDECA7
:10497700D39D4019906F40120048E493FC906F3E1E
:10498700120048E49390008012716BECF0AE59AFBF
:104997005A742D6F4E7006755A33755900AE59AF5C
:1049A7005A74022FFF50010E8E598F5A785A74018C
:1049B70026F6500418E436F640030248FD22755ADD
:1049C70000755900AE59AF5A7432BE00039F5003A9
:1049D700024A92906F71120048E49390008012711E
:1049E7006B0FBF00010EE0FC906F71120048ECFEE8
:1049F700E493FFEEC39F5026AE59AF5A0FBF000195
:104A07000E906F71120048AE59AF5AE493FC906F45
:104A170071120048E49390008012716BECF0AE596C
:104A2700AF5A906F71120048E49390008012716B37
:104A3700E0FC906F73120048ECFCE493FDECD39D0F
:104A47004019906F73120048E493FC906F71120045
:104A570048E49390008012716BECF0AE59AF5A7432
:104A67002D6F4E7006755A33755900AE59AF5A748B
:104A7700022FFF50010E8E598F5A785A740126F66D
:104A8700500418E436F640030249CB2275A7108577
:104A9700F97385FA747E017F00E57412713AE57344
:104AA7002FFF50010E8E598F5AAC5BAD5CEF2DFD79
:104AB700EE3CFC8C5B8D5C123DF5123E00123E0B0A
:104AC7009000C8E0D394024009123E16123E21120C
:104AD7003E2C75A7002285F97385FA747E017F0045
:104AE700E57412713AE5732FFF50010E8E598F5AF4
:104AF7007E017F76900105E012713AAC59AD5AED0F
:104B07002FFFEC3EFE8E5B8F5CE55CF5EDE55BF51C
:104B1700EE90006DE4F0741290004BF02285F9736B
:104B270085FA747E017F00E57412713AE5732FFFF1
:104B370050010E8E598F5A900014E0FCA3E0FDEF50
:104B47002DFDEE3CFC8C5B8D5CE55CF5FDE55BF5D6
:104B5700FE22056422A2DBB340089000D4E0900057
:104B67006DF0A2DCB34048A2965006741990004B32
:104B7700F0A2955006741990004BF0A2A05006744D
:104B87001990004BF0A2975006741990004BF0A2B1
:104B9700A25006741990004BF0A2A1500674199008
:104BA700004BF0C296C295C2A0C297C2A2C2A1751D
:104BB700D8402285A77275A7109000C8E0D3940249
:104BC70050079000E6E0B40252A2D8B34002C29365
:104BD700A2D9B34002C294A2DAB34002C2919000B4
:104BE700C8E0640260079000C8E0B40417A2DBB312
:104BF7004002C292A2DCB34002C287A2DDB34002E8
:104C0700C2908015A2D8B34002C292A2D9B3400283
:104C1700C287A2DAB34002C290802DA2D8B3400A5D
:104C2700C2939000E6E06002C292A2D9B3400AC2E2
:104C3700949000E6E06002C287A2DAB3400AC2910C
:104C47009000E6E06002C29075D8408572A7229076
:104C5700F800E4936406600280FE12009E75A700C8
:104C670075D80075D90475DD0975DE0975D84075E5
:104C7700A71075D80075D90475DA0975DB0975DCD5
:104C87000975DD0975DE0975DF0975D84075A70057
:104C97001200FB7509C875080012062475A70FE5F1
:104CA700FC90005AF0E5FB90005BF0E5FA90005CA1
:104CB700F0E5F990005DF075A70090F800E493F532
:104CC70027120743900897E0D3940350079008975B
:104CD700E0B401067400900897F0900897E09008F8
:104CE700EEF074019000C9F0900897E09069A1F880
:104CF700282873802A802875A70F75F30F75A700DA
:104D0700A2A3400674029000C9F0801375A70F751F
:0F4D1700F31775A700A2A4400674029000C9F01C
:0C69A100024CFA024CFC024CFE024D13AA
:104D26009000C9E0B4022AC218120AEC740290007C
:104D3600C9F0900897E09069ADF828287380108034
:0F4D46000E74009000D8F0800674009000E5F025
:0C69AD00024D43024D45024D47024D4F84
:104D55008028D218120A0174019000C9F0900897B2
:104D6500E09069B9F82828738010800E74009000CF
:0A4D7500D8F0800674009000E5F00D
:0C69B900024D6D024D6F024D71024D79D0
:104D7F0090F807E493900067F0900067E044089084
:104D8F000067F0900067E054FE900067F01203BDDB
:104D9F00123EE89008A4E090016CF09008A5E09016
:104DAF00016DF09008A6E090016EF090016CE0703C
:104DBF000C90016DE0700690016EE060028004C2FD
:104DCF00208002D2209000BAE004900071F0900190
:104DDF0024E0B4FF067400900124F0900125E0B4A4
:104DEF00FF067400900125F012473490F802E49307
:104DFF00B405051248F7801290F802E493D3940596
:104E0F00400512482980031249C574009000F0F044
:104E1F00124030E5B54401F5B5740690004DF074BD
:104E2F000090004EF0740190004FF090F802E49360
:104E3F00900050F090F803E493900051F090F80434
:104E4F00E493900052F07406900053F0900050E0FD
:104E5F00B405067405900053F0900050E0B40406BA
:104E6F007404900053F07431900054F07403900068
:104E7F0055F07407900056F07401900057F090F8B9
:104E8F0005E493900058F090F806E493900059F0E1
:104E9F007400900061F07400900062F07400900054
:104EAF0063F07400900064F07400900065F074007B
:104EBF00900066F074FF900068F0A2B6B39206A25D
:104ECF00B3B39207A2A4B3921DA2A3B3921E9000F4
:104EDF0069E4F0756F00743A900780F074FD9007E5
:104EEF0081F090006AE4F0756E0190004BE4F09051
:104EFF0000CAE0B40106741A90004BF0C21C75632F
:104F0F0000C20BD20CC202757100C21F1205C6750A
:104F1F005F00756B007561007565327566007567AA
:104F2F0000756800756900756A0090001AE4F0A3B7
:104F3F00F0756C00D2B2D2A4D2B0D2B1D2A3D2A7A4
:104F4F00D2A6D2A5D2B77E017F009000A7E0127142
:104F5F003A9000A6E02FFF50010E900024EEF0A330
:104F6F00EFF0EFD394FFEE940F4007900024E4F09E
:104F7F00A3F09000EFE0700674FF9000EFF0900048
:104F8F00CAE07005756D028003756D0374009001A2
:104F9F000FF07400900110F074299006C6F074158C
:104FAF0090076EF0741690076FF07417900770F0FB
:104FBF007400900774F07400900775F074019007F7
:104FCF0076F07402900777F07403900778F074000E
:104FDF0090077CF0740090077DF0D29CE570D3941D
:104FEF001040037570109006C7E0D3940C40067400
:104FFF00009006C7F09006CBE0D3940C40067400E7
:10500F009006CBF09006CFE0D3940C40067400903E
:10501F0006CFF09006D3E0D3940C400674009006B0
:10502F00D3F09006D7E0D3940C400674009006D7C7
:10503F00F09006DBE0D3940C400674009006DBF092
:10504F009006DFE0D3940C400674009006DFF090DA
:10505F0006E3E0D3940C400674009006E3F090064C
:10506F00E7E0D3940C400674009006E7F0D2EC759D
:10507F00CF01A298B34005C298120C54E54D6006BB
:10508F00A299B3B340028005C2991210E0E54E64B5
:10509F00016005E54EB4040280D5C28E7E107F00FC
:1050AF00E56412713AE58D75F010A4FDACF0EF2DAB
:1050BF00FDEE3CFCE58B75F01084FF7E00ED2FFFBD
:1050CF00EC3EFE8E538F54D28E9000ADE060569022
:1050DF00001C12714890001CE0FCA3E0FD90001E24
:1050EF00E0FAA3E0FBEDB5033CECB50238B216A233
:1050FF0003B34013A216B34008E5B54404F5B580D9
:10510F0006E5B554FBF5B590001EE0FEA3E0FF9059
:10511F000020E0FCA3E0FDEF2DFDEE3CFC90001E17
:10512F00ECF0A3EDF09000BAE060099000BAE0C394
:10513F00940340030251EB123027A2034008900062
:10514F00A4E0F545801BE55FC395605005754500EC
:10515F00800F900091E0C3956150069000B7E0F585
:10516F0045E54575F002A4FFAEF090088CEEF0A374
:10517F00EFF0AC2EAD2FEDD39FEC9E402CE5B55448
:10518F00BFF5B59006C7E07006E5B554F7F5B590D5
:10519F0000BAE0B402099000D8E0C3940240028044
:1051AF0006E5B54480F5B58033900069E0C39411EE
:1051BF00502AE5B54440F5B59006C7E07006E5B551
:1051CF004408F5B59000BAE0B402099000D8E0C3E6
:1051DF00940240028006E5B5547FF5B59000BAE021
:1051EF00B40324123142AE2EAF2F90088CE0FCA3F3
:1051FF00E0FDEFD39DEE9C4008E5B54440F5B5804A
:10520F0006E5B554BFF5B5900095E06009A2B3303F
:10521F000701B3B34002805AA2B3300701B3405223
:10522F00A2B3300901B3403DA209B39207E56D70F7
:10523F000FA2B6B3B3500990007CE0C394044002B0
:10524F008006740390004BF0A2B6B3400590007C2B
:10525F00E4F090007CE004F090007CE0B40506746C
:10526F000590004BF0A209B330B301B34004A2097B
:10527F009207A2B6300601B350030257B9A2B63057
:10528F000601B350030257B9A2B6300801B3500359
:10529F000256F1756E00A2B3B3B35006A205B3B3B5
:1052AF0040028006740590004BF0A2B39205055E94
:1052BF00A2B3B3B35006A20AB3B3400302538EE5B1
:1052CF006DB4032EA223B34022E55EB40403756DC3
:1052DF0001E55EC39404500690004B7401F0E55E47
:1052EF00D394044006740290004BF0755E01D223F4
:1052FF008062E56DB40206756D01755E04E55EB4FE
:10530F000405755E01804D90004BE07038E55EC37B
:10531F009404500690004B7401F0E55ED394044062
:10532F0006740290004BF0E55EC394045002D21C49
:10533F00E55ED394044002D21CC296C295C2A0C2AD
:10534F0097C2A2C2A19000CAE0B4010512464B80D9
:10535F0003755E0174029008EAF0A21A9219A20472
:10536F00B34005A21AB39219C204A2A4B34002C259
:10537F001DA2A3B34002C21EA21CB34002C21CE571
:10538F006DC394035006E55E6404600280067404E6
:10539F0090004BF09000C8E0B40308900043E06524
:1053AF005E6002800BA219B34004D21B8002C21BA5
:1053BF00E55EB403499000ADE0604390001CE0FE51
:1053CF00A3E0FF9000ADE08E048F05FF12712A74E9
:1053DF00018C068D07120039900020EEF0A3EFF03C
:1053EF00900020E0F8A3E090001EC8F0A3C8F09052
:1053FF00001CE4F0A3F0C216E5B554FBF5B5AE57AB
:10540F00AF58AC53AD54EF2DFDEE3CFC8C578D587F
:10541F00AE53AF54EFD39DEE9C4011900012E0FAC3
:10542F00A3E0FBEBC394E8EA9403400280069000EC
:10543F001212714890000CE553F0A3E554F0900060
:10544F000EE553F0A3E554F0AE53AF54740C8E0435
:10545F008F05FF12712A8C558D56C28E758D007572
:10546F008B00756400755401755300D28E90000C3B
:10547F00E0FEA3E0FFEF4E600B7CAC7D6012702866
:10548F008E518F52AE51AF527428BE00039F5010F1
:10549F00E5632FFF50010E74011200398E518F52A8
:1054AF008552639000D1E0A851B8000DD3955240BA
:1054BF0008E55290004AF080099000D1E014900066
:1054CF004AF0E56D6006755200755100E55E6401A6
:1054DF006005E55EB403099000BAE06003122CDDAD
:1054EF00E56FB41303756F00A20B500302566A9059
:1054FF0000D6E0C394045006A20AB3B3400302558A
:10550F00B5900086E0B40173900108E0B402141264
:10551F00128190006EE075F0BCA4FFAEF08E5B8F31
:10552F005C8056E56775F00A84FF7E009005801257
:10553F000048E0F55A755900AE59AF5A9000ABE0EC
:10554F0012713A74648E048F05FF12712A8C5B8D71
:10555F005CE55C900046F0AE59AF5A900084E012C3
:10556F00713A74648E048F05FF12712A74BC8C0615
:10557F008D0712713A8E5B8F5C8017900084E075F7
:10558F00F0BCA4FFAEF08E5B8F5C9000ABE09000A0
:10559F0046F0E561C394CC5006E55C455B70028034
:1055AF0003124A93D20B9000D6E0B404069008EA97
:1055BF00E0700302566A900086E0B4017390010810
:1055CF00E0B4021412128190006EE075F0BCA4FFDB
:1055DF00AEF08E5B8F5C8056E56775F00A84FF7EB8
:1055EF0000900580120048E0F55A755900AE59AF8A
:1055FF005A9000ABE012713A74648E048F05FF125B
:10560F00712A8C5B8D5CE55C900046F0AE59AF5A09
:10561F00900084E012713A74648E048F05FF12714A
:10562F002A74BC8C068D0712713A8E5B8F5C8017C3
:10563F00900084E075F0BCA4FFAEF08E5B8F5C90A1
:10564F0000ABE0900046F0E561C394CC5006E55CFA
:10565F00455B70028003124A93D20BE56DB40106CD
:10566F00A20AB3B34002800975700090004C740118
:10567F00F0E56D70689000CDE0600D90006DE0A8D2
:10568F0051B800069552400280299000CDE0B40237
:10569F0008757003756C00800CC200756C0090006B
:1056AF001AE4F0A3F090006DE06006740990004BCF
:1056BF00F0802A757000900040E0B55E0690004CB7
:1056CF007401F0900041E0B55E06740290004CF05A
:1056DF00900042E0B55E06740390004CF0A208B350
:1056EF009206A208B330B601B350030257B9756ED4
:1056FF0001E5B54401F5B5740B900069F0A208926D
:10570F0006E55ED394484014D20AE55ED3944D402B
:10571F000B740590004BF0D21C755E469000D5E0DF
:10572F00B40107E56AC3944140028018E56AC39447
:10573F00145008741390004BF08006740E90004BB9
:10574F00F012464B900053E0FE900050E0C39E4095
:10575F0009900050E0D39408400974FB90004BF07F
:10576F0012464B900051E06015900051E0FE900002
:10577F004FE06E600974FC90004BF012464B9000A6
:10578F0052E06015900052E0FE900054E06E600908
:10579F0074FE90004BF012464B900897E060069015
:1057AF000105E060028003120BD7A21CB3400CC2AC
:1057BF0096C295C2A0C297C2A2C2A1900105E06095
:1057CF000CAE51AF527414BE00059F40028037904B
:1057DF00008DE09069C5F8282873802A8028A2A33D
:1057EF00B35005A21EB340028005124ADDD21E80BF
:1057FF0015A2A4B35005A21DB340028005124ADDC5
:06580F00D21D80028000A2
:1069C5000257E90257EB0257ED025800025813022D
:0269D500581553
:10581500A20DB3B35008900043E0655E60030259E2
:1058250083A201B35006A200B3B3400302597D9091
:1058350000C8E0B404028003025941123D75900886
:10584500EAE0B40202800302592FA21BB34067901D
:105855000119E0601F900018E0FEA3E0FF90011120
:10586500E012713A74C88E048F05FF12712A8C5BA1
:105875008D5C800A900018E0F55BA3E0F55CAE5BFB
:10588500AF5C745E12713A74058E048F05FF127158
:105895002AAE59AF5AED2FFFEC3EFE8E5B8F5C9022
:1058A5000038E0FCA3E0FDEF2DFDEE3CFC8C5B8DAC
:1058B5005C123DF58068900119E0D39403401F9078
:1058C5000018E0FEA3E0FF900114E012713A74C8DD
:1058D5008E048F05FF12712A8C5B8D5C800A900007
:1058E50018E0F55BA3E0F55CAE5BAF5C745E12712E
:1058F5003A74058E048F05FF12712AAE59AF5AED21
:105905002FFFEC3EFE8E5B8F5C900038E0FCA3E041
:10591500FDEF2DFDEE3CFC8C5B8D5C123E16900080
:10592500E6E0B40103123E378010123DF5123E1633
:105935009000E6E0B40103123E378039123D75123E
:105945003DF59000C8E0B4030ED2929000E6E0B4B5
:105955000103123E37801E9000E6E0B40206123DB8
:10596500B7123E169000E6E0B40106A202B3B340BA
:10597500028002D29275A700C20DD20ED20FA20EDE
:10598500B3B35008900044E0655E6003025B04A277
:1059950001B35006A200B3B34003025AFE9000C8FB
:1059A500E0B404028003025AB2123D759008EAE0A1
:1059B500B402028003025AA0A21BB3406A900119E7
:1059C500E0D39401401F900018E0FEA3E0FF900192
:1059D50012E012713A74C88E048F05FF12712A8C79
:1059E5005B8D5C800A900018E0F55BA3E0F55CAE8A
:1059F5005BAF5C745E12713A74058E048F05FF12FD
:105A0500712AAE59AF5AED2FFFEC3EFE8E5B8F5CCF
:105A1500900038E0FCA3E0FDEF2DFDEE3CFC8C5B37
:105A25008D5C123E008068900119E0D39404401FFC
:105A3500900018E0FEA3E0FF900115E012713A74A2
:105A4500C88E048F05FF12712A8C5B8D5C800A90CD
:105A55000018E0F55BA3E0F55CAE5BAF5C745E122D
:105A6500713A74058E048F05FF12712AAE59AF5A2B
:105A7500ED2FFFEC3EFE8E5B8F5C900038E0FCA3C3
:105A8500E0FDEF2DFDEE3CFC8C5B8D5C123E219024
:105A950000E6E0B40103123E378010123E00123ECC
:105AA500219000E6E0B40103123E378049123D75AE
:105AB500123E009000E6E0C394025007A202B340F4
:105AC50002D2879000C8E0B4030ED2879000E6E0CA
:105AD500B40103123E37801E9000E6E0B4020612C0
:105AE5003DB7123E219000E6E0B40106A202B3B331
:105AF50040028002D28775A700D20DC20ED20FA236
:105B05000FB3B35008900045E0655E6003025C8505
:105B1500A201B35006A200B3B34003025C7F90001C
:105B2500C8E0B404028003025C33123D759008EAB4
:105B3500E0B402028003025C21A21BB3406A90011B
:105B450019E0D39402401F900018E0FEA3E0FF90F7
:105B55000113E012713A74C88E048F05FF12712A81
:105B65008C5B8D5C800A900018E0F55BA3E0F55C2A
:105B7500AE5BAF5C745E12713A74058E048F05FFDF
:105B850012712AAE59AF5AED2FFFEC3EFE8E5B8F98
:105B95005C900038E0FCA3E0FDEF2DFDEE3CFC8CB5
:105BA5005B8D5C123E0B8068900119E0D394054033
:105BB5001F900018E0FEA3E0FF900116E012713A75
:105BC50074C88E048F05FF12712A8C5B8D5C800A68
:105BD500900018E0F55BA3E0F55CAE5BAF5C745E2E
:105BE50012713A74058E048F05FF12712AAE59AFF2
:105BF5005AED2FFFEC3EFE8E5B8F5C900038E0FC8B
:105C0500A3E0FDEF2DFDEE3CFC8C5B8D5C123E2C84
:105C15009000E6E0B40103123E378010123E0B12ED
:105C25003E2C9000E6E0B40103123E378049123D58
:105C350075123E0B9000E6E0C394025007A202B332
:105C45004002D2909000C8E0B4030ED2909000E6D6
:105C5500E0B40103123E37801E9000E6E0B4020670
:105C6500123DB7123E2C9000E6E0B40106A202B345
:105C7500B340028002D29075A700D20DD20EC20F9A
:0D5C8500E5709069D7F82828739000EDE0D5
:0369D700025C8ED1
:105C9200906A64F828287312260C801212260C804F
:0E5CA2000D1226968008122742800312274218
:0F6A6400025C99025C9E025CA3025CA8025CAD1E
:105CB0007570010260E412286E1229857570020267
:105CC00060E4122D21A203B340139000D2E075F0DE
:105CD0001DA4FFAEF0900014EEF0A3EFF09008804A
:105CE000E0FEA3E0FF741412713A90000EE0FCA3F2
:105CF000E0FD74068F02FF12712A8D078C038E045B
:105D00008A058B06127028900884EEF0A3EFF090BD
:105D100000D6E0B401087446BE00059F4002800D25
:105D20007446900884F8E4F0E8A3F0801B9008849F
:105D3000E0FEA3E0FF74F0BE00039F500B74F090F0
:105D40000884F8E4F0E8A3F0E536700375360190B6
:105D50000884E0FEA3E0FFE5362FFF50010E900817
:105D600084EEF0A3EFF0757003A22A401A90004C65
:015D7000E052
:0669DA00025CB6025CC283
:105D7100906A73F8282873800D75700A8008757011
:065D81000B800375700C9D
:0C6A7300025D78025D7A025D7F025D84A6
:105D87000260E49006C7E060077401F508122E4F21
:105D9700A22CB3B3500890077EE0642A6002800902
:105DA700E5B54402F5B5025E519000BBE0D394021D
:105DB700404590008FE02403A851B8000495525045
:105DC70009900091E0D395615002800ED201A22282
:105DD7004006740890004BF0D22290008FE0A85143
:105DE700B80005D39552500B900091E02403C3955A
:105DF700615002C201805390008FE02403A851B87C
:105E0700000495525010E55FC395605009900091CA
:105E1700E0D395615002800ED201A2224006740899
:105E270090004BF0D22290008FE0A851B80005D324
:105E370095525014E560240FC3955F400B90009175
:105E4700E02403C395615002C201A2014002C222AD
:105E5700A22CB3500DA201B3500890077EE0642A2C
:105E670060028006E5B554FDF5B59000D5E07007F2
:105E7700E56AC3941440028002D2019000CAE0B4DC
:105E87000102D201A2014005757004800A757010E5
:0E5E970090001AE4F0A3F00260E49000BBE07B
:0669E000025D8A025EA1C7
:105EA500906A7FF82828731213978012121397802F
:0E5EB5000D12154A8008121601800312160104
:0F6A7F00025EAC025EB1025EB6025EBB025EC09A
:105EC3009006CBE060077402F508122E4F7570053B
:105ED3000260E412175A7570069006CFE0600774EB
:105EE30003F508122E4F9006D3E060077404F508FB
:105EF300122E4F0260E4900046E06006A203B3B3A3
:105F03004002800DE55ED394015006900046E014F4
:105F1300F01219E37570079006D7E060077405F572
:105F230008122E4F9006DBE060077406F508122E68
:105F33004F0260E4900108E0B40203121308121E3A
:105F43004B7570089006DFE060077407F508122EA2
:105F53004F9006E3E060077408F508122E4F0260C5
:105F6300E4121F2D7570090260E4122305A20DB31C
:105F73005005A20EB340028006D20DD20ED20F7589
:105F830070109006E7E060077409F508122E4F02BF
:105F930060E490003BE0C39446500AC296C29774F3
:105FA3004690003BF085365A755900900040E0F565
:105FB30073123FC6E55C90003BF0900006E559F094
:105FC300A3E55AF0C211900884E0F559A3E0F55A0D
:105FD300900040E0F573123FC6E55C90003AF09004
:105FE3000000E559F0A3E55AF0C210E56DB40105D0
:105FF30075700B80037570030260E490003DE0C38D
:10600300944650139000D6E0B40102C296C295C2E2
:10601300A2744690003DF085365A755900900041B0
:10602300E0F573123FC6E55C90003DF0900008E593
:1060330059F0A3E55AF0C213900884E0F559A3E0A0
:10604300F55A900041E0F573123FC6E55C90003CC1
:10605300F0900002E559F0A3E55AF0C212E56DB4E1
:10606300010575700C8003757003807590003FE027
:10607300C3944650139000D6E0B40102C296C2A066
:10608300C2A1744690003FF085365A7559009000BE
:1060930042E0F573123FC6E55C90003FF090000AC2
:1060A300E559F0A3E55AF0C215900884E0F559A329
:1060B300E0F55A900042E0F573123FC6E55C9000AC
:1060C3003EF0900004E559F0A3E55AF0C214E56DE3
:1060D300B40103756D00757003800680048002802F
:0160E30000BC
:1069E600025ED6025EF9025F37025F64025F6D02E5
:1069F6005F95025FFE02606F0260DE0260E0026089
:046A0600E20260E464
:1060E40090003AE0B55E028003026198A210406B12
:1060F400900000E0FEA3E0FFEF4E605DAC51AD52B6
:10610400740ABC0033D39D402FAA55AB5674058A3C
:10611400048B05FF12712A8D068C07900000E0FCA9
:10612400A3E0FDCFCECF120003740112003990001A
:1061340000EEF0A3EFF08021AE55AF56900000E0E2
:10614400FCA3E0FD120003740A8E048F05FF127194
:106154002A900000ECF0A3EDF0D210AE53AF5490AF
:106164000000E0FCA3E0FDEFC39DEE9C4026124B33
:10617400249000D6E0906A0AF8282873800ED296FC
:0C618400800AD2968006D296D297800046
:0F6A0A0002618002618202618602618A026190EC
:10619000C21074C890003AF0A210B3B35007900038
:1061A0003AE0B55E028026124B249000D6E0906A59
:1061B00019F8282873800ED296800AD2968006D2CB
:0561C00096D29780005B
:0F6A19000261B50261B70261BB0261BF0261C5D4
:1061C50074C890003AF0C21090003BE0B55E0280C2
:1061D50003026267A211406B900006E0FEA3E0FF98
:1061E500EF4E605DAC51AD52740ABC0033D39D4097
:1061F5002FAA55AB5674058A048B05FF12712A8D9B
:10620500068C07900006E0FCA3E0FDCFCECF120080
:10621500037401120039900006EEF0A3EFF080211F
:10622500AE55AF56900006E0FCA3E0FD12000374E6
:106235000A8E048F05FF12712A900006ECF0A3ED7B
:10624500F0D211AE53AF54900006E0FCA3E0FDEF91
:10625500C39DEE9C400CC296C297744690003BF0DD
:10626500C211A211B3B3500790003BE0B55E0280A6
:106275000CC296C297744690003BF0C21190003C48
:10628500E0B55E028003026336A212406B90000205
:10629500E0FEA3E0FFEF4E605DAC51AD52740ABC69
:1062A5000033D39D402FAA55AB5674058A048B0540
:1062B500FF12712A8D068C07900002E0FCA3E0FD19
:1062C500CFCECF1200037401120039900002EEF018
:1062D500A3EFF08021AE55AF56900002E0FCA3E09D
:1062E500FD120003740A8E048F05FF12712A9000B7
:1062F50002ECF0A3EDF0D212AE53AF54900002E0E1
:10630500FCA3E0FDEFC39DEE9C4026124B249000BC
:10631500D6E0906A28F8282873800ED296800AD293
:09632500958006D295D2A28000F9
:0F6A280002631E02632002632402632802632EAE
:10632E00C21274C890003CF0A212B3B35007900092
:10633E003CE0B55E028026124B249000D6E0906AB7
:10634E0037F8282873800ED296800AD2958006D20E
:05635E0095D2A28000B1
:0F6A370002635302635502635902635D02636396
:1063630074C890003CF0C21290003DE0B55E02801C
:106373000302640EA213406B900008E0FEA3E0FF4B
:10638300EF4E605DAC51AD52740ABC0033D39D40F7
:106393002FAA55AB5674058A048B05FF12712A8DFB
:1063A300068C07900008E0FCA3E0FDCFCECF1200DF
:1063B300037401120039900008EEF0A3EFF080217E
:1063C300AE55AF56900008E0FCA3E0FD1200037445
:1063D3000A8E048F05FF12712A900008ECF0A3EDDA
:1063E300F0D213AE53AF54900008E0FCA3E0FDEFEE
:1063F300C39DEE9C40159000D6E0B40102C296C244
:1064030095C2A2744690003DF0C213A213B3B350D9
:106413000790003DE0B55E0280159000D6E0B40120
:1064230002C296C295C2A2744690003DF0C2139078
:10643300003EE0B55E0280030264E6A214406B9066
:106443000004E0FEA3E0FFEF4E605DAC51AD52747B
:106453000ABC0033D39D402FAA55AB5674058A045A
:106463008B05FF12712A8D068C07900004E0FCA3B4
:10647300E0FDCFCECF120003740112003990000467
:10648300EEF0A3EFF08021AE55AF56900004E0FC90
:10649300A3E0FD120003740A8E048F05FF12712A14
:1064A300900004ECF0A3EDF0D214AE53AF5490007F
:1064B30004E0FCA3E0FDEFC39DEE9C4026124B24B9
:1064C3009000D6E0906A46F8282873800ED2968012
:0B64D3000AD2A08006D2A0D2A1800057
:0F6A46000264CE0264D00264D40264D80264DE1B
:1064DE00C21474C890003EF0A214B3B350079000DB
:1064EE003EE0B55E028026124B249000D6E0906A04
:1064FE0055F8282873800ED296800AD2A08006D234
:05650E00A0D2A18000F5
:0F6A550002650302650502650902650D026513FE
:1065130074C890003EF0C21490003FE0B55E028064
:10652300030265BEA215406B90000AE0FEA3E0FFE4
:10653300EF4E605DAC51AD52740ABC0033D39D4045
:106543002FAA55AB5674058A048B05FF12712A8D49
:10655300068C0790000AE0FCA3E0FDCFCECF12002B
:1065630003740112003990000AEEF0A3EFF08021CA
:10657300AE55AF5690000AE0FCA3E0FD1200037491
:106583000A8E048F05FF12712A90000AECF0A3ED26
:10659300F0D215AE53AF5490000AE0FCA3E0FDEF38
:1065A300C39DEE9C40159000D6E0B40102C296C292
:1065B300A0C2A1744690003FF0C215A215B3B35018
:1065C3000790003FE0B55E0280159000D6E0B4016D
:1065D30002C296C2A0C2A1744690003FF0C21590B9
:1065E30000D8E0B40202800302670A90006BE0D394
:1065F3009566506490006BE0F4042566FE9000DB22
:10660300E08E00F5F0E884FF7E008F73EFC39410F3
:10661300500CEF8573F0A4FDACF08D73800375739C
:10662300FF90006BE0D39573400B90006BE0C39534
:1066330073F57180037571009000F6E0D395714096
:10664300069000F6E0F5719000F7E0C395715006EF
:106653009000F7E0F571807190006BE0C39566FEE2
:106663009000DBE08E00F5F0E884FF7E008F73EF8F
:10667300C39410500CEF8573F0A4FDACF08D7380C0
:10668300037573FF85735A75590090006BE0255AA3
:10669300FFAE5950010E8E598F5A74FFBE0009D3B5
:1066A3009F4005855A7180037571FF9000F6E0D312
:1066B300957140069000F6E0F5719000F7E0C39500
:1066C3007150069000F7E0F571A203B3B3500D903B
:1066D300006CE0FE9000E3E0D39E5002800E74074E
:1066E30090004BF0E5B554BFF5B5801B75A710E5D9
:1066F300CDC395714008E5B554BFF5B58006E5B542
:106703004440F5B575A7009000F3E0605E9000FD8E
:10671300E0A851B80004955250179000FCE0A8512E
:10672300B8000ED3955240099000FEE0D395614026
:1067330002801D75A710E5CDC394BF4008E5B5548D
:10674300EFF5B58006E5B54410F5B575A700801BD8
:1067530075A710E5CDC394404008E5B554EFF5B5F2
:106763008006E5B54410F5B575A7009000F4E06028
:106773005E900100E0A851B80004955250179000B4
:10678300FFE0A851B8000ED395524009900101E0F3
:10679300D395614002801D75A710E5CDC394BF401A
:1067A30008E5B554DFF5B58006E5B54420F5B575C4
:1067B300A700801B75A710E5CDC394404008E5B53D
:1067C30054DFF5B58006E5B54420F5B575A700E5BA
:1067D3006FC39413501DE56F75F00284AFF07E0014
:1067E300EF4E70051232FC800AA2EDB34005C2EDF4
:1067F3001232FCAE53AF547450C39F74C39E400C0B
:1068030090006AE0C3945A400302697DA20AB34030
:106813000912464B740690004BF0A20CB3500EE5E0
:1068230061D394334007E561C394CC400280419027
:106833000108E0B4021412128190006EE075F05E5C
:10684300A4FFAEF08E5B8F5C800F900084E075F048
:106853005EA4FFAEF08E5B8F5CE55C455B6011E58B
:10686300B54401F5B5740B900069F0124A93D20C4C
:1068730090006AE0D394014007E561C3941A400293
:106883008002C20C9006C7E060077401F508122E5F
:106893004F9006CBE060077402F508122E4F900666
:1068A300CFE060077403F508122E4F9006D3E06023
:1068B300077404F508122E4F9006D7E0600774059D
:1068C300F508122E4F9006DBE060077406F50812F8
:1068D3002E4F9006DFE060077407F508122E4F90E5
:1068E30006E3E060077408F508122E4F9006E7E010
:1068F30060077409F508122E4F90006AE0C3945A9A
:106903005010E56FB4130990006AE004F0756F004E
:10691300803FE56FB41303756F00C28E758D0075EC
:106923008B00756400755401755300D28E90006915
:10693300E0C394115008900069E004F080067411DC
:10694300900069F0900069E0B41106E5B554FEF5D6
:10695300B590006AE0D394014007E56AC3944140CF
:10696300028006740E90004BF0900897E06006904A
:0D6973000105E060028003120BD702507E88
:106A8E000000010001400160018001A001C001E091
:106A9E0002000300039603B603D603F404000500B8
:106AAE000512052405360548055A056C057E059028
:106ABE0005A805C005DE0600061406280646066E65
:106ACE0006AE05CF06EE00FF013F015F017F019F7D
:106ADE0001BF01DF01FF02FF039503B503D503F3E9
:106AEE0003FF04FF05110523053505470559056B01
:106AFE00057D058F05A705BF05CE05F106130627F3
:106B0E000645066D06AD06ED05DD06FF0FAA0FA5BF
:106B1E000F9F0F9A0F940F8D0F870F800F780F71A5
:106B2E000F680F600F570F4E0F450F3B0F300F259D
:106B3E000F1A0F0E0F020EF50EE80EDB0ECC0EBE68
:106B4E000EAE0E9F0E8E0E7D0E6C0E5A0E470E342E
:106B5E000E200E0C0DF70DE20DCB0DB50D9D0D8516
:106B6E000D6D0D540D3A0D200D050CE90CCE0CB12A
:106B7E000C940C760C580C3A0C1B0BFB0BDB0BBB62
:106B8E000B9A0B790B570B350B130AF10ACE0AAB86
:106B9E000A870A640A400A1C09F809D409B0098C4C
:106BAE0009670943091F08FB08D608B2088E086A50
:106BBE000846082307FF07DC07B907960773075136
:106BCE00072F070D06EC06CA06AA068906690649AE
:106BDE00062A060A05EC05CD05B005920575055881
:106BEE00053C0520050504EA04CF04B5049C048287
:106BFE000469045104390422040B03F403DE03C8B0
:106C0E0003B2039D038903750361034D033B032800
:106C1E000316030402F202E102D102C002B002A086
:106C2E00029102820273026502570249023C022F50
:106C3E0002220216020901FD01F201E601DB01D07A
:106C4E0001C601BB01B101A7019D0194018B018217
:106C5E00017901700168016001580150014801413C
:106C6E0001390132012B0125011E01180111010B01
:106C7E00010500FF00FA0FA60FA00F990F920F8BC0
:106C8E000F840F7C0F740F6B0F620F580F4E0F4354
:106C9E000F380F2C0F1F0F120F050EF70EE80ED820
:106CAE000EC80EB70EA50E930E800E6C0E580E4229
:106CBE000E2C0E150DFD0DE40DCB0DB10D950D79B0
:106CCE000D5D0D3F0D200D010CE10CC00C9E0C7CDA
:106CDE000C590C350C100BEA0BC40B9E0B760B4F9C
:106CEE000B260AFD0AD40AAA0A800A550A2A09FFA7
:106CFE0009D409A8097C0950092508F908CD08A16D
:106D0E000875084A081E07F307C8079D0773074949
:106D1E00072006F706CE06A6067E06570630060A9A
:106D2E0005E405BF059B057705540532051004EFF4
:106D3E0004CE04AE048F047104530435041903FD0C
:106D4E0003E203C703AD0394037B0363034B0334D6
:106D5E00031E030802F302DE02CA02B602A3029168
:106D6E00027F026D025C024C023C022C021D020EDE
:106D7E00020001F201E401D701CA01BE01B101A670
:106D8E00019A018F0185017A01700166015D01533F
:106D9E00014A014101390131012901210119011273
:106DAE00010B010400FD00F700F000EA00E400DE34
:106DBE0000D900D300CE00C900C400BF00BA00B590
:106DCE0000B100AD00A800A400A0009C00990095A1
:106DDE000091008E008A008700840081007E007B77
:10009E0075B50075840175A70075FFA075EF069004
:1000AE000047E4F075C91075A70F75A1C775A700B5
:1000BE0075D90075CE0C75A70F75F1FE75F2FF752B
:1000CE00F30775F47875A4BA75A5FF75A60775AE16
:1000DE000075AFFF75D48175D5FF75D6FF75D7FF47
:1000EE0075A70075A20175A14775F8092275E60876
:1000FE0075E71075BC0175BE0475BD6C75BE0775D0
:10010E00BDA075BE0875BD0175BC0075BB1875BC6C
:10011E002075BA0875E88075D11375A70F75E105BE
:10012E0075E20075C74012464B759700759780743F
:10013E000A12711A7597C0E5975420700280F875EF
:10014E008F0275A700D2AF75980075A90C75A70F11
:10015E0075AB4375ADFB75AC1E75A71075C91875DB
:10016E00CA0075CB0075C80475A700758912758E07
:10017E0004758C00758A00C2A9D28C758D00758BA2
:10018E0000D2ABD28E75B62075D944C2992290009A
:10019E0082E0900896F090008DE0900897F0900025
:1001AE008EE0900898F09000ADE0900899F09000E5
:1001BE00BAE090089AF09000C8E090089BF090008A
:1001CE00D6E090089CF09000D8E090089DF090004A
:1001DE00E6E090089EF09000F3E090089FF090000B
:1001EE00F4E09008A0F0900106E09008A1F09001D4
:1001FE001EE09008A3F090016CE09008A4F090012E
:10020E006DE09008A5F090016EE09008A6F09001C8
:10021E0005E09008A7F09000EFE09008A8F090009D
:10022E00A6E09008A9F09000A7E09008AAF0900030
:10023E00A1E09008ABF09000A2E09008ACF0900125
:10024E000BE09008ADF090010CE09008AEF090013C
:10025E000DE09008AFF090010EE09008B0F0900124
:10026E000FE09008B1F09006C6E09008B2F090064C
:10027E00CAE09008B3F09006CEE09008B4F0900675
:10028E00D2E09008B5F09006D6E09008B6F0900651
:10029E00DAE09008B7F09006DEE09008B8F090062D
:1002AE00E2E09008B9F09006E6E09008BAF0900609
:1002BE00EAE09008BBF090076EE09008BCF0900763
:1002CE006FE09008BDF0900770E09008BEF09007C8
:1002DE0071E09008BFF0900772E09008C0F09007B0
:1002EE0073E09008C1F0900774E09008C2F0900798
:1002FE0075E09008C3F0900776E09008C4F0900780
:10030E0077E09008C5F0900778E09008C6F0900767
:10031E0079E09008C7F090077AE09008C8F090074F
:10032E007BE09008C9F090077CE09008CAF0900737
:10033E007DE09008CBF090077EE09008CCF0900125
:10034E0010E09008CDF0900111E09008CEF09001F1
:10035E0012E09008CFF0900113E09008D0F09001D9
:10036E0014E09008D1F0900115E09008D2F09001C1
:10037E0016E09008D3F0900117E09008D4F09001A9
:10038E0018E09008D5F0900119E09008D6F0900092
:10039E00B4E09008D7F09000ECE09008D8F090010F
:1003AE0024E09008D9F0900125E09008DAF0229030
:1003BE000896E0900082F0900897E090008DF09003
:1003CE000898E090008EF0900899E09000ADF090C3
:1003DE00089AE09000BAF090089BE09000C8F09068
:1003EE00089CE09000D6F090089DE09000D8F09028
:1003FE00089EE09000E6F090089FE09000F3F090E9
:10040E0008A0E09000F4F09008A1E0900106F090B2
:10041E0008A3E090011EF09008A7E0900105F0906F
:10042E0008A8E09000EFF09008A9E09000A6F090E8
:10043E0008AAE09000A7F09008ABE09000A1F09021
:10044E0008ACE09000A2F09008ADE090010BF090A7
:10045E0008AEE090010CF09008AFE090010DF09026
:10046E0008B0E090010EF09008B1E090010FF0900E
:10047E0008B2E09006C6F09008B3E09006CAF0907D
:10048E0008B4E09006CEF09008B5E09006D2F09059
:10049E0008B6E09006D6F09008B7E09006DAF09035
:1004AE0008B8E09006DEF09008B9E09006E2F09011
:1004BE0008BAE09006E6F09008BBE09006EAF090ED
:1004CE0008BCE090076EF09008BDE090076FF090CA
:1004DE0008BEE0900770F09008BFE0900771F090B2
:1004EE0008C0E0900772F09008C1E0900773F0909A
:1004FE0008C2E0900774F09008C3E0900775F09082
:10050E0008C4E0900776F09008C5E0900777F09069
:10051E0008C6E0900778F09008C7E0900779F09051
:10052E0008C8E090077AF09008C9E090077BF09039
:10053E0008CAE090077CF09008CBE090077DF09021
:10054E0008CCE090077EF09008CDE0900110F0907E
:10055E0008CEE0900111F09008CFE0900112F090DB
:10056E0008D0E0900113F09008D1E0900114F090C3
:10057E0008D2E0900115F09008D3E0900116F090AB
:10058E0008D4E0900117F09008D5E0900118F09093
:10059E0008D6E0900119F09008D7E09000B4F090E2
:1005AE0008D8E09000ECF09008D9E0900124F0908B
:1005BE0008DAE0900125F02275470090088EE4F0ED
:1005CE00A3F0753100753000754D00754E00C226D2
:1005DE00D227900897E06002D21F74FE900890F820
:1005EE00E4F0E8A3F074FE900894F8E4F0E8A3F0C9
:1005FE0074FE900892F8E4F0E8A3F0745A9008E8BC
:10060E00F0745A9008E9F0D228C224C22AC229C234
:10061E0025C22CC23222750B00750A00AE0AAF0B32
:10062E00AC08AD09EDC39FEC9E401674FF12711A13
:10063E0075CF01780B740126F6500418E436F65087
:10064E00DB22C2AF75D904758F0375B7A575B7F1E7
:10065E0090F800E4F0758F0175B7A575B7F1E52731
:10066E0090F800F075B7A575B7F190F801E4F07544
:10067E00B7A575B7F19008DCE090F802F075B7A554
:10068E0075B7F19008E0E090F803F075B7A575B76F
:10069E00F19008DDE090F804F075B7A575B7F1900C
:1006AE0008DEE090F805F075B7A575B7F19008DF94
:1006BE00E090F806F075B7A575B7F19008E1E090F7
:1006CE00F807F0758F0075D944D2AF22900047E03D
:1006DE00B4AB61C2AF75D90475B62275F522758FAC
:1006EE000375B7A575B7F1740090F600F0758F011C
:1006FE00755A00755900AE59AF5A7445BE00279F02
:10070E00402475B7A575B7F1900896120048E0FC25
:10071E0090F600120048ECF0785A740126F6500458
:10072E0018E436F650D0758F0075F51175B6207534
:10073E00D944D2AF22C2AF75F52275D904755A00CD
:10074E00755900AE59AF5A7445BE00229F401F9096
:10075E00F600120048E493FC900896120048ECF064
:10076E00785A740126F6500418E436F650D575D929
:10077E004475F511D2AF22900047E0B4AA0280036F
:10078E000208C2C2AF75D90475B62275F522758FEF
:10079E000375B7A575B7F1740090F400F075B7A5A1
:1007AE0075B7F1740090F200F075B7A575B7F174D6
:1007BE000090F000F075B7A575B7F1740090EE00DB
:1007CE00F0758F01755A00755900AE59AF5A74FF06
:1007DE00C39F74019E402475B7A575B7F190008034
:1007EE00120048E0FC90F400120048ECF0785A74C5
:1007FE000126F6500418E436F650CF755A00755996
:10080E0000AE59AF5A74FFC39F74019E402475B752
:10081E00A575B7F1900280120048E0FC90F200122C
:10082E000048ECF0785A740126F6500418E436F6B7
:10083E0050CF755A00755900AE59AF5A74FFC39F09
:10084E0074019E402475B7A575B7F190048012000F
:10085E0048E0FC90F000120048ECF0785A74012643
:10086E00F6500418E436F650CF755A00755900AE9E
:10087E0059AF5A74FFC39F74019E402475B7A57576
:10088E00B7F1900680120048E0FC90EE001200488E
:10089E00ECF0785A740126F6500418E436F650CF70
:1008AE00758F0075F51175B62075D944D2AF743AAF
:1008BE00900780F022900047E0B4AA028003020A5B
:1008CE0000C2AF75D90475B62275F522758F037502
:1008DE00B7A575B7F1740090EC00F075B7A575B7B4
:1008EE00F1740090EA00F075B7A575B7F174009039
:1008FE00E800F075B7A575B7F1740090E600F075D5
:10090E008F01755A00755900AE59AF5A74FFC39FC7
:10091E0074019E402475B7A575B7F1900080120042
:10092E0048E0FC90EC00120048ECF0785A74012676
:10093E00F6500418E436F650CF755A00755900AECD
:10094E0059AF5A74FFC39F74019E402475B7A575A5
:10095E00B7F1900280120048E0FC90EA00120048C5
:10096E00ECF0785A740126F6500418E436F650CF9F
:10097E00755A00755900AE59AF5A74FFC39F740172
:10098E009E402475B7A575B7F1900480120048E01B
:10099E00FC90E800120048ECF0785A740126F650EC
:1009AE000418E436F650CF755A00755900AE59AF9B
:1009BE005A74FFC39F74019E402475B7A575B7F195
:1009CE00900680120048E0FC90E600120048ECF021
:1009DE00785A740126F6500418E436F650CF758F07
:1009EE000075F51175B62075D944D2AF743A9007DB
:1009FE0080F022C2AF75D90475F522755A0075596B
:100A0E0000AE59AF5A74FFC39F74019E401F90F4FD
:100A1E0000120048E493FC900080120048ECF0783D
:100A2E005A740126F6500418E436F650D4755A005E
:100A3E00755900AE59AF5A74FFC39F74019E401F83
:100A4E0090F200120048E493FC900280120048ECF1
:100A5E00F0785A740126F6500418E436F650D47520
:100A6E005A00755900AE59AF5A74FFC39F74019E58
:100A7E00401F90F000120048E493FC900480120096
:100A8E0048ECF0785A740126F6500418E436F65005
:100A9E00D4755A00755900AE59AF5A74FFC39F747E
:100AAE00019E401F90EE00120048E493FC900680D9
:100ABE00120048ECF0785A740126F6500418E43609
:100ACE00F650D475F51175D944D2AF74019000C9A2
:100ADE00F0743A900780F09008EF7401F022C2AFE4
:100AEE0075D90475F522755A00755900AE59AF5A6D
:100AFE0074FFC39F74019E401F90EC00120048E4E7
:100B0E0093FC900080120048ECF0785A740126F69F
:100B1E00500418E436F650D4755A00755900AE5983
:100B2E00AF5A74FFC39F74019E401F90EA001200DB
:100B3E0048E493FC900280120048ECF0785A74015D
:100B4E0026F6500418E436F650D4755A007559003E
:100B5E00AE59AF5A74FFC39F74019E401F90E800B8
:100B6E00120048E493FC900480120048ECF0785A8E
:100B7E00740126F6500418E436F650D4755A0075F2
:100B8E005900AE59AF5A74FFC39F74019E401F9017
:100B9E00E600120048E493FC900680120048ECF048
:100BAE00785A740126F6500418E436F650D475F5CA
:100BBE001175D944D2AF74029000C9F0743A9007FF
:100BCE0080F074029008EFF02274019000C9F0904A
:100BDE000897E0903CBBF828287380188016A2A3D3
:100BEE00400674029000C9F0800AA2A44006740266
:040BFE009000C9F0AA
:0C3CBB00020BE8020BEA020BEC020BF813
:100C02009000C9E0B40105A230B34002801AD2308C
:100C120012464B120A0174019000C9F01203BD1270
:100C22003EE8741B90004BF09000C9E0B40206A2AB
:100C320030B3B34002801AC23012464B120AEC742F
:100C4200029000C9F01203BD123EE8741B90004BE3
:100C5200F022E54E64046006E59964FF600280318B
:100C6200A2264004D2268027E54E600874E6254E6F
:100C720090004BF0E54D600874F0254D90004BF06C
:100C8200E54EB4010280FE754E00754D00C226800D
:100C920002C226E54E903CC7F8282873754E00E53F
:100CA20099B4FF03754D01E599B4FE03754D02E554
:100CB20099B4FD03754D03E599B4FC03754D04E544
:100CC20099B4FA03754D05E599B4FB06754E011208
:100CD200464BE599B4F906754E0412464BE599B4B4
:100CE200F73312464BC29C74AB900047F01206DAFF
:100CF20074AA900047F09008EFE0B401051207854E
:100D020080031208C3900047E4F0D29C754E007530
:100D12004D007599F7E599D394E54007E599C39499
:100D2200F04002801685994F754E027E017F00E5E4
:100D32004FC394E612713A8E328F3390088EE4F0EC
:100D4200A3F0E599D394C24007E599C394E6400223
:100D5200802885994F754E0374E5C3954FF5337519
:100D62003200AE32AF33906A8E127109E493F87496
:100D7200019390088EC8F0A3C8F0D2990210DF90B8
:100D820008A3E0700AA220B35005A221B34002805A
:100D92005C90088EE0FEA3E0FF74FFBE00039F504C
:100DA20009EFC39446EE9406402B90088EE0FEA312
:100DB200E0FFEFD3946DEE94064009EFC394EEEE9C
:100DC2009406401190088EE0FEA3E0FFEFD394FF5B
:100DD200EE9406401390088EE0FEA3E0FF900080A0
:100DE200120048E599F08003859974801190088E6D
:100DF200E0FEA3E0FF900080120048E599F0900821
:100E02008E12714890088EE0FEA3E0FFEFB4010657
:100E1200EEB407028003020EDA900780E0B43C02CF
:100E22008003020EDAA220B35005A221B340028051
:100E320055C29C1203BD90008DE09008EEF0124066
:100E42003090016CE09008A4F090016DE09008A54C
:100E5200F090016EE09008A6F074AB900047F0129B
:100E620006DA74AA900047F09008EFE0B401051288
:100E7200078580031208C39008EFE09000C9F09044
:100E82000047E4F08047C29C12019C74009008A4C1
:100E9200F074009008A5F074009008A6F090008D00
:100EA200E09008EEF012403074AB900047F012066A
:100EB200DA74AA900047F01207851208C3D29C7513
:100EC20099FB75096475080012062480FED29C7590
:100ED2004E00754D007599FB0210DF90088EE0FE02
:100EE200A3E0FFEF4E700685993175300090088EB1
:100EF200E0FEA3E0FF74016F4E701BAC30AD31AA6F
:100F020032AB33ED2BFBEC3AFA8A068B079000806A
:100F1200120048E599F090088E12714890088EE010
:100F2200FEA3E0FF74026F4E7021AC30AD317456F7
:100F32006D4C7006E54F64E66002800312464B1268
:100F42004030854F99754E00754D000210DF9008B4
:100F52008EE0FEA3E0FF900080120048E599F09039
:100F6200088E12714890088EE0FEA3E0FFAC32AD0D
:100F7200338F028E038C068D07906AD4127109E4B6
:100F820093F9740193FEEAD39EEB994009854F9938
:100F9200754E00754D000210DF90088EE0FEA3E052
:100FA200FF900080120048E599F090088E12714877
:100FB20090088EE0FEA3E0FFEFB40006EEB401025B
:100FC20080030210DF90005DE0D394C7400B9000D5
:100FD2005DE0C394C8F550801A90005DE0D394633D
:100FE200400B90005DE0C39464F550800690005D74
:100FF200E0F550E55075F002A4FFAEF08F73EF906C
:10100200008012716BEFFCE0FDEC90008312716BBB
:10101200EDFCE0FDEC2DB5500280030210D10FEF84
:1010220090008012716BE573FFE0FCEF9000841278
:10103200716BECFFE0FCEFC39CB550028003021021
:10104200D1E57390008212716BE573FFE0FCEF90C3
:10105200008512716BECFFE0FCEF2CB55071E5736B
:1010620090008612716BE0C395509008DCF0E57336
:1010720090008712716BE0C395509008DDF0E57324
:1010820090008A12716BE0C395509008DEF0E57310
:1010920090008B12716BE0C395509008DFF0E573FE
:1010A20090008C12716BE0C395509008E0F0E573EC
:1010B20090008D12716BE0C395509008E1F012061A
:1010C200507599F975096475080012062480FE7539
:0D10D20099FF75096475080012062480FE60
:0F3CC700020C9E020D81020EDD020F50020F9BB8
:1010DF0022E54D903CD6F82828730211C490088E53
:1010EF00E0FEA3E0FF90004D120048E0F599900854
:1010FF008E12714890088EE0FEA3E0FF741C6F4EB5
:10110F007003754D000211C4856E990211C49008C9
:10111F008EE0FEA3E0FF900080120048E0F599EF0B
:10112F00B40107EEB40703754D0090088E12714895
:07113F000211C490088FE0CB
:0F3CD6000210E90210EC02111702111D02114237
:10114600903D48F82828738552998067855F998075
:1011560062856199805D8565998058856799805318
:10116600856899804E8569998049856A99804490F9
:10117600001BE0F599803CA227B340077599FAC297
:10118600278017A21FB3400575990F800B90004B5F
:10119600E0F59990004BE4F0C21F8017856B9980AB
:1011A60012856699800D856C9980087599FC800377
:0311B600754D0074
:103D480002114D02115202115702115C0211610257
:103D5800116602116B02117002117502117D0211B8
:0D3D6800A20211A70211AC0211B10211B6A6
:0B11B90090088E1271488003123F4323
:033CE5000211C108
:1011C40022E537255AFFAE5950010E9000801200D7
:1011D40048E0F538E537255AFFAE5950010E0FBFE8
:1011E40000010E900080120048E0F539853F3BE590
:1011F40038B539058538378041E539D39538401DF0
:10120400E539C39538853AF0A4FFAEF0E53B8E048A
:101214008F05FF12712AED2538F537801DE538C397
:101224009539853AF0A4FFAEF0E53B8E048F05FFB7
:1012340012712AEDF4042538F53722E539D39538AF
:10124400401DE539C39538853AF0A4FFAEF0E53B7F
:101254008E048F05FF12712AED2538F537801DE5C0
:1012640038C39539853AF0A4FFAEF0E53B8E048F80
:1012740005FF12712AEDF4042538F5372290008613
:10128400E0B4017FE56775F00A84FF7E008F37E5DF
:101294006775F00A84ADF07C008D3A753F0A755984
:1012A40005755A24E537C3941150051211C58006FB
:1012B4009005B5E0F537E537C394F05008E537906D
:1012C400006EF0800674EF90006EF0E56775F00A2A
:1012D40084FF7E008F37E56775F00A84ADF07C00EB
:1012E4008D3A753F0A755905755A5AE537C39411F5
:1012F40050051211C580069005EBE0F537E53790EF
:101304000046F022900086E0B401028003021396A6
:10131400E56775F00A84FF7E008F37E56775F00A8C
:1013240084ADF07C008D3A753F0A755905755A36BF
:10133400E537C3941150051211C580069005C7E026
:10134400F537E537C394F0500585374B8003754B6B
:10135400EFE56775F00A84FF7E008F37E56775F067
:101364000A84ADF07C008D3A753F0A755905755AAB
:1013740048E537C3941150051211C580069005D96C
:10138400E0F537E537C394F0500585374C80037595
:101394004CEF22E55F75F00484FF7E008F37E55F34
:1013A40075F00484ADF07C008D3A753F04755901E5
:1013B400755A00E537C3943F50051211C580069055
:1013C40001BFE0F537E537900888F8E4F0E8A3F0CA
:1013D40090004AE075F020A4FFAEF09000D1E08EBA
:1013E400048F05FF12712A8D379000B9E0D3955F01
:1013F40050030214A29000DDE0D3955F4010ED90FD
:1014040001C012716BE0F52B752A0002149F900045
:10141400A8E0D3955F4043E5379001C012716BE0BB
:10142400F538E5379001E012716BE0F5399000DD95
:10143400E0F404255FF53A9000A8E0FE9000DDE0BA
:10144400F4042EF53BE538B53905853837800312A9
:10145400123F85372B752A008041E5379001E01251
:10146400716BE0F538E53790020012716BE0F539E5
:101474009000A8E0F404255FF53A9000B9E0FE90EE
:1014840000A8E0F4042EF53BE538B5390585383776
:10149400800312123F85372B752A000215499000EC
:1014A400E0E0D3955F5011E53790024012716BE094
:1014B400F52B752A000215499000A9E0D3955F50D9
:1014C40043E53790022012716BE0F538E53790025E
:1014D4004012716BE0F5399000A9E0F404255FF542
:1014E4003A9000E0E0FE9000A9E0F4042EF53BE51C
:1014F40038B53905853837800312123F85372B7587
:101504002A008041E53790020012716BE0F538E55E
:101514003790022012716BE0F5399000B9E0F404C1
:10152400255FF53A9000A9E0FE9000B9E0F4042E9E
:10153400F53BE538B53905853837800312123F8508
:10154400372B752A00229000F1E0F53C753F1175A8
:101554005902755A00AE51AF52E53C75F00FA4FD27
:10156400ACF0EDD39FEC9E4021E53C8E048F05FF4B
:1015740012712AED75F010A4FFAEF0E55F75F0115D
:1015840084FD7C00ED2FF53D800EE55F75F0118440
:10159400FF7E00EF24F0F53D853D37E55F75F011E2
:1015A40084AFF07E008F3A1211C585373EAE51AF3D
:1015B400529000F1E075F00FA4FDACF0EDD39FEC78
:1015C4009E4028755902755A10853D371211C585FC
:1015D4003E38853739AE51AF52E53C8E048F05FF56
:1015E4001271558D3A853C3B12123FE537900888BD
:1015F400F8E4F0E8A3F0752B64752A00229000F15A
:10160400E0F53C753F11755902755A00AE51AF5261
:10161400E53C75F00FA4FDACF0EDD39FEC9E4021AA
:10162400E53C8E048F05FF12712AED75F010A4FFBE
:10163400AEF0E56175F01184FD7C00ED2FF53D8081
:101644000EE56175F01184FF7E00EF24F0F53D8511
:101654003D37E56175F01184AFF07E008F3A1211C9
:10166400C585373EAE51AF529000F1E075F00FA43E
:10167400FDACF0EDD39FEC9E4028755902755A10CD
:10168400853D371211C5853E38853739AE51AF5285
:10169400E53C8E048F05FF1271558D3A853C3B1253
:1016A400123FE537900888F8E4F0E8A3F0E56B60B2
:1016B40017E56BC394FE50109000E5E0B402099066
:1016C40000D3E0D3940B5002801F900888E0FEA35F
:1016D400E0FFE56B12713A74E78E048F05FF127117
:1016E4002A900888ECF0A3EDF09000BBE0B4045F0E
:1016F400E55F75F00484FF7E008F37E55F75F004C5
:1017040084ADF07C008D3A753F04755901755A001B
:10171400E537C3943F50051211C580069001BFE020
:10172400F537900888E0FEA3E0FFE53712713A74BC
:10173400328E048F05FF12712A900888E0FEA3E020
:10174400FFEF2DFDEE3CFC900888ECF0A3EDF07566
:101754002B64752A0022900086E0B40146E5677583
:10176400F00A84FF7E008F37E56775F00A84ADF0D8
:101774007C008D3A753F0A755905755A00E537C3E3
:10178400941150051211C58006900591E0F537AE0D
:101794002AAF2BE5372FFF50010E746412717D8E32
:1017A4002A8F2B900087E0B40146E56875F00A841F
:1017B400FF7E008F37E56875F00A84ADF07C008DFC
:1017C4003A753F0A755905755A6CE537C39411503B
:1017D400051211C580069005FDE0F537AE2AAF2B42
:1017E400E5372FFF50010E746412717D8E2A8F2B02
:1017F400900096E0B40249E56AC3944175F005840B
:10180400FF7E008F37E56A75F00584ADF07C008DAE
:101814003A753F05755906755A00E537C394135058
:10182400051211C58006900693E0F537AE2AAF2B5A
:10183400E5372FFF50010E746412717D8E2A8F2BB1
:101844009000D8E0B4020280030218F9E55F75F055
:101854001584FF7E008F37E55F75F01584ADF07C4D
:10186400008D3A753F15755903755AF4E537C394DD
:101874000B50051211C5800690047FE0F537E5375B
:1018840075F0FFA4FFAEF09000D9E08E048F05FF41
:1018940012712AED90006BF0E56675F078A4FFAE46
:1018A400F074FF8E048F05FF12712A8C598D5A74BF
:1018B400028C068D071200398F37AC59AD5A740467
:1018C400FF1271558D3A753F04755906755A28E50E
:1018D40037C3941D50051211C580069006C5E0F566
:1018E40037AE2AAF2BE5372FFF50010E7464127107
:1018F4007D8E2A8F2B900085E0B4025DE56175F042
:1019040064A4FFAEF074081200398E5B8F5C74051A
:101914008E048F05FF12712A8D37AE5BAF5C7405A0
:101924008E048F05FF1271558D3A753F0575590563
:10193400755ADEE537C3941350051211C58006901D
:101944000671E0F537AE2AAF2BE5372FFF50010EB5
:10195400746412717D8E2A8F2B9000C7E0707F9083
:10196400004AE075F00A84FF7E008F3790004AE059
:1019740075F00A84ADF07C008D3A753F0A755905FF
:10198400755AC0E537C3940E50051211C5800690F0
:10199400064EE0F537E53790006FF09000E6E0B4CE
:1019A400023C90004AE075F00A84FF7E008F379075
:1019B400004AE075F00A84ADF07C008D3A753F0A68
:1019C400755905755ACFE537C3940E50051211C5E4
:1019D400800690065DE0F537E537900070F02290C0
:1019E400008EE0B401179008E3E0252BFFAE2A50E7
:1019F400010E9000E2E012717D8E2A8F2B90010679
:101A0400E0B40114900107E0A851B80004955250C5
:101A140007E55FC39560400280139000B0E0252B7A
:101A2400FFAE2A50010E8E2A8F2B021E4A90008E82
:101A3400E0B40306A224B3B3400280509008EDE062
:101A440070109008E6E0C39405A851B800069552BA
:101A5400400280109000B0E0252BFFAE2A50010E0A
:101A64008E2A8F2B9008EDE0600D9008E6E0A851D7
:101A7400B800069552400280109000B0E0252BFF7C
:101A8400AE2A50010E8E2A8F2B021E4A900088E047
:101A9400B402028003021E4A90008BE0602FE567C7
:101AA400D394464028900012E0FEA3E0FF9000C6C5
:101AB400E075F003A4FDACF0EFD39DEE9C400E90D6
:101AC40000EAE0A851B80005D395525003021E4A1B
:101AD4009000BBE0B403028003021C9285615A7536
:101AE4005900900092E0A851B800049552500E900D
:101AF4000093E0A859B80005D3955A5003021C8FEF
:101B0400E56175F002A4FFAEF074158E048F05FF35
:101B140012712A8C068D07900610120048FEE0FF11
:101B2400EE90008AE0FEEF8E0088F0A4FFAEF07421
:101B3400648E048F05FF12712A8C598D5A90004AC5
:101B4400E075F018A4FFAEF09000D1E08E048F058C
:101B5400FF12712A8C068D07900628120048AE5990
:101B6400AF5AE012713A74648E048F05FF12712A21
:101B74008C598D5AE565A859B80005D3955A500378
:101B8400021C06E565C3955AFFE49559FE8E598FEC
:101B94005A7428BE00039F500C755A287559007456
:101BA4000D90004BF0AE59AF5A90008BE012713A91
:101BB40074288E048F05FF12712A8C598D5A90084F
:101BC40088E0FEA3E0FF740A8E048F05FF12712AD9
:101BD4008D068C07AC59AD5ACFCECF120003740AD0
:101BE4008E048F05FF12712A8C598D5A900888E053
:101BF400FEA3E0FF127185900888EEF0A3EFF002D7
:101C04001C8FE565A859B80004955A507EAE59AFAB
:101C14005AE56512717D8E598F5A7428BE00039F50
:101C2400500C755A28755900740D90004BF0AE593C
:101C3400AF5A90008BE012713A74288E048F05FF1E
:101C440012712A8C598D5A900888E0FEA3E0FF7423
:101C54000A8E048F05FF12712A8D068C07AC59ADCC
:101C64005ACFCECF120003740A8E048F05FF12716F
:101C74002A8C598D5A900888E0FEA3E0FFEF2DFDD1
:101C8400EE3CFC900888ECF0A3EDF0021E4A9000B4
:101C9400D3E0855FF0A4FFAEF0740512713A7407C7
:101CA4001200398E598F5A900092E0A851B800045E
:101CB40095525012900093E075F002A4FDACF0EF41
:101CC400C39DEE9C4003021E4AE55F75F00B84FF42
:101CD4007E00900610120048FEE0FFEE90008AE0BD
:101CE400FEEF8E0088F0A4FFAEF074648E048F05BE
:101CF400FF12712A8C598D5A90004AE075F018A48D
:101D0400FFAEF09000D1E08E048F05FF12712A8C93
:101D1400068D07900628120048AE59AF5AE012719A
:101D24003A74648E048F05FF12712A8C598D5AE51A
:101D340065A859B80005D3955A5003021DC1E5653D
:101D4400C3955AFFE49559FE8E598F5A7428BE00E4
:101D5400039F500C755A28755900740D90004BF070
:101D6400AE59AF5A90008BE012713A74288E048FEA
:101D740005FF12712A8C598D5A900888E0FEA3E061
:101D8400FF740A8E048F05FF12712A8D068C07AC2E
:101D940059AD5ACFCECF120003740A8E048F05FFBB
:101DA40012712A8C598D5A900888E0FEA3E0FF1224
:101DB4007185900888EEF0A3EFF0021E4AE565A84D
:101DC40059B80004955A507EAE59AF5AE565127160
:101DD4007D8E598F5A7428BE00039F500C755A2863
:101DE400755900740D90004BF0AE59AF5A90008BAA
:101DF400E012713A74288E048F05FF12712A8C59EF
:101E04008D5A900888E0FEA3E0FF740A8E048F05C3
:101E1400FF12712A8D068C07AC59AD5ACFCECF1262
:101E24000003740A8E048F05FF12712A8C598D5A8F
:101E3400900888E0FEA3E0FFEF2DFDEE3CFC900847
:101E440088ECF0A3EDF0229000E6E0B4027BE55FBD
:101E540075F00884FF7E008F37E55F75F00884AD68
:101E6400F07C008D3A753F08755901755AE0E537E5
:101E7400C3943F50051211C5800690027FE0F537E8
:101E8400E53790088AF8E4F0E8A3F090088AE0FEC9
:101E9400A3E0FFAC2AAD2B12000374648E048F05FB
:101EA400FF12712A90088AECF0A3EDF0900083E011
:101EB4008C068D0712713A74648E048F05FF1271BB
:101EC4002A90088AECF0A3EDF0900888E0FEA3E0E5
:101ED400FFAC2AAD2B12000374648E048F05FF122D
:101EE400712A900888ECF0A3EDF0900083E08C0652
:101EF4008D0712713A74648E048F05FF12712A9053
:101F04000888ECF0A3EDF0A203401DAE51AF52746B
:101F140005BE00039F5002D203E561D394CC400870
:101F2400D201741190004BF0229000E5E0B4020855
:101F34009000D3E0640B60028045900888E0FEA323
:101F4400E0FFE56B12713A74E78E048F05FF12719E
:101F54002A900888ECF0A3EDF09000E6E0B4021FAC
:101F640090088AE0FEA3E0FFE56B12713A74E78EF5
:101F7400048F05FF12712A90088AECF0A3EDF0900B
:101F840000A5E05402601B90009CE0A851B8001228
:101F9400D39552400DA203B3B35007E561C3949A9D
:101FA4004002805FAE34AF3590009AE075F002A431
:101FB400FDACF0EF2DFDEE3CFC74022DFD50010C48
:101FC400E561BC003ED39D403A754301A22B4033EA
:101FD40090009BE075F05EA4FDACF07405FF1271F7
:101FE4002A8C5B8D5C124A93900888E0FEA3E0FF84
:101FF40090009BE02FFF50010E900888EEF0A3EFB5
:10200400F0D22BE561A834B8000495355002C22BF8
:10201400856135753400E54370030221239000F88F
:10202400E0C395435003022115900108E0C39402D4
:1020340040030220BFE56775F00A84FF7E00900527
:1020440080120048E0F55A755900AE59AF5A900015
:102054009BE012713A74648E048F05FF12712A8C0E
:102064005B8D5C9000F8E004C395438C068D0712E9
:10207400713A9000F8E08E048F05FF12712A8C5B90
:102084008D5C900888E0FEA3E0FFEF2DFDEE3CFCA4
:10209400900888ECF0A3EDF09000E6E0B4021A900A
:1020A400088AE0FEA3E0FFAA5BAB5CEF2BFBEE3AF1
:1020B400FA90088AEAF0A3EBF080569000F8E00466
:1020C400C39543854BF0A4FFAEF09000F8E08E0476
:1020D4008F05FF12712A8C5B8D5C900888E0FEA34B
:1020E400E0FFEF2DFDEE3CFC900888ECF0A3EDF052
:1020F4009000E6E0B4021A90088AE0FEA3E0FFAA8A
:102104005BAB5CEF2BFBEE3AFA90088AEAF0A3EBA8
:10211400F005439000F8E0C39543500375430090E5
:1021240000A5E05401601B900099E0A851B800128A
:10213400D39552400DA203B3B35007E55FC394CCCB
:1021440040028060900097E075F003A4FFAEF0E5D4
:10215400402FFF50010E74032FFF50010EE55FBEA8
:102164000042D39F403E754401A22B403790009813
:10217400E075F05EA4FFAEF074058E048F05FF12C7
:10218400712A8C5B8D5C124A93900888E0FEA3E070
:10219400FF900098E02FFF50010E900888EEF0A306
:1021A400EFF0D22BE55FC395405002C22B855F4010
:1021B400E54470030222BD9000F9E0C39544500346
:1021C4000222AF900108E0C394024003022259E5C1
:1021D4006775F00A84FF7E00900580120048E0F5E0
:1021E4005A755900AE59AF5A900098E012713A747A
:1021F400648E048F05FF12712A8C5B8D5C9000F94C
:10220400E004C395448C068D0712713A9000F9E0FE
:102214008E048F05FF12712A8C5B8D5C900888E018
:10222400FEA3E0FFEF2DFDEE3CFC900888ECF0A34C
:10223400EDF09000E6E0B4021A90088AE0FEA3E014
:10224400FFAA5BAB5CEF2BFBEE3AFA90088AEAF04C
:10225400A3EBF080569000F9E004C39544854CF05C
:10226400A4FFAEF09000F9E08E048F05FF12712AEE
:102274008C5B8D5C900888E0FEA3E0FFEF2DFDEE03
:102284003CFC900888ECF0A3EDF09000E6E0B4028A
:102294001A90088AE0FEA3E0FFAA5BAB5CEF2BFB7D
:1022A400EE3AFA90088AEAF0A3EBF005449000F9BC
:1022B400E0C395445003754400900888E0FEA3E011
:1022C400FF9000AAE0BE00039F500D9000AAE0908A
:1022D4000888F8E4F0E8A3F09000E6E0B402129075
:1022E400088AE0FEA3E0FF9000AAE0BE00059F403C
:1022F40002800D9000AAE090088AF8E4F0E8A3F0C8
:10230400229000E6E0B401028003022453A203B346
:10231400500302243A9000B1E0B4017A900888E0B6
:10232400FEA3E0FFAC51AD52120003743C8E048F47
:1023340005FF12712A9000C1E0BC00159D40129067
:102344000888E0FEA3E0FF9000C3E0BE00039F50B6
:1023540002D202900888E0FEA3E0FFAC51AD521215
:102364000003743C8E048F05FF12712A9000C1E0B3
:10237400C3940ABC001AD39D4016900888E0FEA3BB
:10238400E0FF9000C3E0C39405BE0004D39F500255
:102394008002C202807A900888E0FEA3E0FFAC517C
:1023A400AD5212000374788E048F05FF12712A90C7
:1023B40000C1E0BC00159D4012900888E0FEA3E037
:1023C400FF9000C3E0BE00039F5004D202804190FE
:1023D4000888E0FEA3E0FFAC51AD5212000374780C
:1023E4008E048F05FF12712A9000C1E0C3940ABCC9
:1023F400001AD39D4016900888E0FEA3E0FF9000E9
:10240400C3E0C39405BE0004D39F50028002C202FD
:10241400A202B34021900888E0FEA3E0FF9000C22E
:10242400E012713A74648E048F05FF12712A9008C9
:1024340088ECF0A3EDF0A202B3400CA22F40067486
:102444002490004BF0D22FA2024002C22F8002C27D
:1024540002900046E06006A203B3B34002801990E4
:102464000888E0FEA3E0FF900046E02FFF50010E35
:10247400900888EEF0A3EFF0A200B34006A201B3E7
:10248400B3500990001AE4F0A3F0802D900888E07E
:10249400FEA3E0FF7400D39F74019E40119008884E
:1024A400E0F8A3E090001AC8F0A3C8F0800B74FF12
:1024B40090001AF8E4F0E8A3F09000C8E0C3940494
:1024C400400C9008EAE0C3940240030225AD90005A
:1024D400B1E0B40147900888E0FEA3E0FF745E1207
:1024E400713A74058E048F05FF12712A900888ECE6
:1024F400F0A3EDF09000E6E0B4021F90088AE0FE3D
:10250400A3E0FF745E12713A74058E048F05FF1206
:10251400712A90088AECF0A3EDF08045900888E0D9
:10252400FEA3E0FF745E12713A740A8E048F05FFF5
:1025340012712A900888ECF0A3EDF09000E6E0B464
:10254400021F90088AE0FEA3E0FF745E12713A74E1
:102554000A8E048F05FF12712A90088AECF0A3ED0D
:10256400F0900888E0FEA3E0FF7402BE000CD39F45
:102574004008752902752800800A900888E0F5282B
:10258400A3E0F52990088AE0FEA3E0FF7402BE00F0
:102594000CD39F4008752D02752C00800A90088A80
:1025A400E0F52CA3E0F52D8046900888E0FEA3E03A
:1025B400FF7401BE000CD39F4008752901752800E3
:1025C400800A900888E0F528A3E0F52990088AE0BD
:1025D400FEA3E0FF7401BE000CD39F4008752D01DB
:1025E400752C00800A90088AE0F52CA3E0F52D9064
:1025F4000018E528F0A3E529F0A232B34009C2008F
:1026040090001AE4F0A3F02290004AE090038012B4
:10261400716BE0F54175426490004AE0FE9000BCA5
:10262400E0D39E4037E55F75F00884FF7E008F3766
:10263400E55F75F00884ADF07C008D3A753F087550
:102644005903755A96E537C3941F50051211C58076
:1026540006900435E0F5378537428035E55F75F03F
:102664000884FF7E008F37E55F75F00884ADF07C49
:10267400008D3A753F08755903755AB6E537C3940A
:102684001F50051211C58006900455E0F5378537B3
:1026940042229000F2E0F53C753F11755904755AD9
:1026A40000AE51AF52E53C75F00FA4FDACF0EDD394
:1026B4009FEC9E4021E53C8E048F05FF12712AEDAC
:1026C40075F010A4FFAEF0E55F75F01184FD7C0099
:1026D400ED2FF53D800EE55F75F01184FF7E00EF70
:1026E40024F0F53D853D37E55F75F01184AFF07E4C
:1026F400008F3A1211C585373EAE51AF529000F2A9
:10270400E075F00FA4FDACF0EDD39FEC9E4028756E
:102714005904755A10853D371211C5853E388537E1
:1027240039AE51AF52E53C8E048F05FF1271558DC1
:102734003A853C3B12123F85374175426422900032
:10274400F2E0F53C753F11755904755A00AE51AF6E
:1027540052E53C75F00FA4FDACF0EDD39FEC9E4028
:1027640021E53C8E048F05FF12712AED75F010A44B
:10277400FFAEF0E56175F01184FD7C00ED2FF53DB1
:10278400800EE56175F01184FF7E00EF24F0F53DC5
:10279400853D37E56175F01184AFF07E008F3A1204
:1027A40011C585373EAE51AF529000F2E075F00F7F
:1027B400A4FDACF0EDD39FEC9E4028755904755AE6
:1027C40010853D371211C5853E38853739AE51AF76
:1027D40052E53C8E048F05FF1271558D3A853C3BC2
:1027E40012123F8537417542649000EDE0B40479DC
:1027F40090004AE0FE9000BCE0D39E4037E55F7550
:10280400F00884FF7E008F37E55F75F00884ADF033
:102814007C008D3A753F08755903755A96E537C3A0
:10282400941F50051211C58006900435E0F53785D4
:1028340037428035E55F75F00884FF7E008F37E509
:102844005F75F00884ADF07C008D3A753F087559CA
:1028540003755AB6E537C3941F50051211C5800697
:10286400900455E0F53785374222900086E0B401A4
:102874003BE56775F00A84FF7E008F37E56775F0E6
:102884000A84ADF07C008D3A753F0A755905755A76
:1028940012E537C3941150051211C580069005A3A3
:1028A400E0F537E5422537C39464F542900087E0AC
:1028B400B4013BE56875F00A84FF7E008F37E56854
:1028C40075F00A84ADF07C008D3A753F0A755905A0
:1028D400755A7EE537C3941150051211C5800690D0
:1028E400060FE0F537E5422537C39464F542E54128
:1028F4002542F53690008EE0B402109008E2E025FF
:1029040036FE9000E2E0F4042EF5369000E5E0D3C4
:1029140094014040E56BC394E7501D74E7C3956B85
:10292400FE9008E4E08E00F5F0E884FF7E008F3727
:10293400E5362537F536801CE56BC394E7FE900831
:10294400E4E08E00F5F0E884FF7E008F37E536C3BF
:102954009537F536A2034006E5412464F536E5369D
:10296400D394644009E536C39464F5368003753620
:10297400009000BEE0C3953650069000BEE0F536E8
:1029840022D20090006DE0A851B800049552503E48
:1029940090006DE0A851B800049552500375360FAD
:1029A40090006DE004A851B80004955250037536A8
:1029B4000790006DE02402A851B80004955250021B
:1029C400C20090006DE06006740990004BF0C22ACA
:1029D4007E017F009000C4E012713A9000D3E08E33
:1029E400048F05FF12712AE55FBC000CD39D4008DB
:1029F400D232740A90004BF0900086E0B401099042
:102A040000C5E0C39567400280159000D7E0A85147
:102A1400B8000495525002C200740B90004BF09021
:102A24000086E0B40107E567C394644002801D900A
:102A3400011DE0600D90011DE0A851B800069552FB
:102A440040028008C200740B90004BF0A2004003C7
:102A5400753600C231900106E0B40114900107E01C
:102A6400A851B8000495525007E55FC39560400231
:102A7400802A9000AFE0D3941D400B9000AFE0C3D8
:102A8400941EF5368003753600A22E400874159006
:102A9400004BF0D231D22ED22C022B7FC22CC22E6C
:102AA40090008EE0B40306A224B3B34003022B7F4C
:102AB4009008E6E0C39405A851B800049552500666
:102AC4009008EDE06002801F9000AFE0D3941D40B9
:102AD4000B9000AFE0C3941EF53680037536007486
:102AE4000C90004BF0D2319008E6E0A851B80004F5
:102AF400955250069008EDE07002801F9000AFE000
:102B0400D3941D400B9000AFE0C3941EF5368003B0
:102B1400753600740C90004BF0D2319008E6E0A8B2
:102B240051B80004955250319000CDE0B40228D23F
:102B34002A9008ECE0FE9008EDE0D39E5006900841
:102B4400EDE0700280099008ECE4F0C22A8006905F
:102B540008ECE004F08002C2009008E6E02405A836
:102B640051B80004955250139000CDE0B4020A907D
:102B740008EDE07002D22A8002C200A229B34027E5
:102B84009000AFE0D3941D400B9000AFE0C3941EBF
:102B9400F5368003753600A22D4006741090004B64
:102BA400F0D22DD2318002C22D85366C9000AFE078
:102BB400D3941D401890007DE02536FE90004AE035
:102BC40075F01E84FC7F00EE2CF5368037A231B3FD
:102BD400401690007DE0FE90004AE075F01E84FCF3
:102BE4007F00EE2CF536801C90007FE02536FE90A9
:102BF400007DE02EFE90004AE075F01E84FC7F000C
:102C0400EE2CF536A232B34005D22A756C00229020
:102C1400004AE075F00584FF7E008F3790004AE09B
:102C240075F00584ADF07C008D3A753F0575590348
:102C3400755AD69000D1E01475F00584FF7E00E546
:102C440037BE00039F50051211C5800BE537900471
:102C54005612716BE0F537E5379008E5F09008E51A
:102C6400E0FE9000C0E0C39E50089000C0E09008D1
:102C7400E5F09000AFE0D3941D401E9008E5E0FE1F
:102C840090007DE02EFE90004AE075F01E84FC7FEB
:102C940000EE2C9008E5F0803FA231B3401890007C
:102CA4007DE0FE90004AE075F01E84FC7F00EE2C6F
:102CB4009008E5F080229008E5E0FE90007FE02E89
:102CC400FE90007DE02EFE90004AE075F01E84FC2C
:102CD4007F00EE2C9008E5F022900086E0B40136E7
:102CE400E56775F00A84FF7E00900580120048E0D5
:102CF400F546E546D394644010E546C3946475F004
:102D04000F84FF7E008F4680037546009000A3E089
:102D14002546F54680069000A3E0F54622E5677552
:102D2400F00A84FF7E00900580120048E0C3946995
:102D34004007E567D3946440559000EDE0C39403E5
:102D44005026900882E0FEA3E0FF7404120039E5E7
:102D54005F12713A740F8E048F05FF12712A900866
:102D640080ECF0A3EDF08024900882E0FEA3E0FF65
:102D74007404120039E56112713A740F8E048F05E0
:102D8400FF12712A900880ECF0A3EDF0800F9008F8
:102D940082E0F8A3E0900880C8F0A3C8F0A2034042
:102DA4001A900882E0FEA3E0FF740312713A7401E2
:102DB400120039900880EEF0A3EFF0900096E0B492
:102DC4000262E56AC3944175F00584FF7E008F3783
:102DD400E56A75F00584ADF07C008D3A753F0575A4
:102DE4005906755A14E537C3941750051211C58056
:102DF400069006A7E0F537900880E0FEA3E0FF7494
:102E04000A8E048F05FF12712AE5378C068D07128E
:102E1400713A740A8E048F05FF12712A900880ECAF
:102E2400F0A3EDF0900880E0FEA3E0FF900886E0B8
:102E3400FCA3E0FDEDD39FEC9E400F900886E0F8E4
:102E4400A3E0900880C8F0A3C8F022E50875F00458
:102E5400A4FFAEF09006C3120048E0903CE8F828C6
:102E64002873804C85527380479000D3E0855FF0CF
:102E7400A4FFAEF074081200398F73803385617338
:102E8400802E8567738029856873802485697380A3
:102E94001F856A73801A856B73801585667380102D
:102EA400856573800B856C73800690001BE0F57359
:103CE800022E66022E68022E6D022E81022E860298
:103CF8002E8B022E90022E95022E9A022E9F022EB5
:073D0800A4022EA9022EAE59
:102EB400E50875F004A4FFAEF09006C4120048E5DE
:102EC4000875F004A4FFAEF0E0FC9006C5120048BB
:102ED400ECFEE0FFEEC39F4003022FBCE50875F053
:102EE40004A4FFAEF09006C3120048E0B40441E528
:102EF4000875F004A4FFAEF09006C5120048E0C3C4
:102F04009573500AE508F50CD39233123E4BE5084D
:102F140075F004A4FFAEF09006C4120048E0D39507
:102F240073400AE508F50CC39233123E4B022FBAE4
:102F3400E50875F004A4FFAEF09006C4120048E062
:102F4400C395735015E50875F004A4FFAEF0900620
:102F5400C5120048E0D395735002800AE508F50CC9
:102F6400D39233123E4BE50875F004A4FFAEF09003
:102F740006C4120048E0D395735015E50875F004B3
:102F8400A4FFAEF09006C5120048E0C39573500A42
:102F9400E508F50CC39233123E4B9006CBE0B40126
:102FA400099000DFE0D395615002800A7402F50CA9
:102FB400C39233123E4B806AE50875F004A4FFAE59
:102FC400F09006C4120048E0D395734015E50875E7
:102FD400F004A4FFAEF09006C5120048E0C3957358
:102FE4004002800AE508F50CC39233123E4BE50813
:102FF40075F004A4FFAEF09006C4120048E0C39537
:10300400734015E50875F004A4FFAEF09006C512F0
:103014000048E0D39573400AE508F50CD3923312C7
:103024003E4B22AE2EAF2F74C9BE000CD39F400876
:10303400782E12718D023141752F01752E00AE511B
:10304400AF52E546BE000DD39F40099000B5E0D3D2
:10305400954740028023754700E546C39552F573B2
:103064009000B8E0D395454008E5452573F54580C3
:10307400069000B8E0F54580020547900091E0D342
:103084009561401CE55FC395604015AE51AF52E5B4
:1030940046BE00039F50099000B6E0D39548400215
:1030A400806E9008E7E0A851B8000495525003756B
:1030B4004A009008E7E0A851B8000BD395524006A7
:1030C400E5529008E7F0E54A7041E552C39546F5AC
:1030D40073E573D3940540037573059000B7E0C39B
:1030E40095455007E573C3954540028009E545C3FE
:1030F4009573F54580069000B7E0F5459000B7E07C
:10310400D3954540069000B7E0F545754800800228
:103114000548E54A7016900091E0C39561500DE5AD
:10312400462405A851B8000695524002800F90002D
:10313400A4E0F545754A0174789008E7F022AE2EB4
:10314400AF2F74E9D39F74039E4008782E12718DBB
:103154000232FB752F01752E00754532A225403DC4
:10316400E54775F00284AFF07E00EF4E70057545BB
:103174001980037545329000A4E075F002A4FFAEF7
:10318400F0E547BE0006D39F4002D2250547754AA5
:103194000374789008E7F07549000232E2AE51AF4B
:1031A40052E5466F4E70030232E2E546BE000DD38F
:1031B4009F40099000B5E0D395474002800F7547C2
:1031C40000E54AC394035003754519800DE546C3D1
:1031D4009552F573E5472573F547900091E0D39533
:1031E40061400E9008E7E0A851B80007D39552401B
:1031F40002800C05499000A4E0B54903754A00E536
:103204004AB40306A203B3B34002800A0549E54960
:10321400B43C03754A02E54AB402299008E7E0A8E1
:1032240051B8000ED395524009E5529008E7F07565
:103234004900900091E0C395615009754900747884
:103244009008E7F0E54A705A900091E0D395614008
:103254001CE55FC395604015AE51AF52E546BE0014
:10326400039F50099000B6E0D3954840028008754A
:10327400480075454B8028E552C39546F573E573C0
:10328400D394054003757305900091E0D395614094
:1032940008E5482573F5488006E5482406F5487591
:1032A4004900E54A7016900091E0C39561500DE520
:1032B400462405A851B80006955240028003754A79
:1032C40001E54AB4011875451905499000A4E0B513
:1032D4004906754A0275490074789008E7F0A2011E
:1032E400B34003754532E54575F00AA4FFAEF0908E
:1032F400088CEEF0A3EFF022E56F903D0FF828283C
:1033040073023CA8900089E0700302362C9000BF41
:10331400E0B4010280030234BF900048E0655E60BF
:1033240009E552455160030234BC7E017F00E5BECD
:1033340012713AE5BD2FFF50010E8E598F5A90013C
:1033440024E075F010A4FDACF08C5B8D5CEFD39D94
:10335400EE9C40091271858E598F5A8006755A0069
:10336400755900AE59AF5A740E12713A9000B4E018
:103374008E048F05FF12712A900890ECF0A3EDF0F3
:10338400E56B600FE56BC394FE50089000E5E064C4
:1033940002600280649000D3E0B40B1F900890E0B8
:1033A400FEA3E0FF74E712713AE56B8E048F05FF0C
:1033B40012712A900890ECF0A3EDF09000D3E0D3C2
:1033C400940B40089000BBE064046002802B9008DA
:1033D40090E0FEA3E0FF900894E0FCA3E0FDEFD3AF
:1033E4009DEE9C400D127185900890EEF0A3EFF0D5
:1033F4008007900890E4F0A3F0900890E0FEA3E02A
:10340400FFEFD39400EE94014008D232742690006A
:103414004BF0A232B3B3502C7E057F009000D3E072
:103424008E048F05FF12712A900890E0FEA3E0FF3E
:10343400EFC39DEE9C400FAC51AD52740FBC000421
:10344400D39D50028002C232900089E0B4022790DA
:103454000892E0FEA3E0FF900890E0FCA3E0FDEFFB
:103464002DFDEE3CFC74018C068D0712003990088A
:1034740090EEF0A3EFF0900890E0FEA3E0FF900838
:1034840092E0FCA3E0FDEDD39FEC9E4004D22880A3
:1034940002B228900890E0F8A3E0900892C8F0A344
:1034A400C8F09000BBE064016006A228B3B34002F8
:1034B4008006900891E0F55F02362AD2287E017FCB
:1034C40000E5BE12713AE5BD2FFF50010E8E598FF3
:1034D4005A900124E075F010A4FDACF08C5B8D5C77
:1034E400EFD39DEE9C40091271858E598F5A800648
:1034F400755A00755900AE59AF5A740E12713A904C
:1035040000B4E08E048F05FF12712A900890ECF04D
:10351400A3EDF0E56B600FE56BC394FE50089000DB
:10352400E5E06402600280649000D3E0B40B1F9075
:103534000890E0FEA3E0FF74E712713AE56B8E0495
:103544008F05FF12712A900890ECF0A3EDF0900023
:10355400D3E0D3940B40089000BBE0640460028085
:103564002B900890E0FEA3E0FF900894E0FCA3E019
:10357400FDEFD39DEE9C400D127185900890EEF006
:10358400A3EFF08007900890E4F0A3F0900890E097
:10359400FEA3E0FFEFD39400EE94014008D232740E
:1035A4002690004BF0A232B3B3502C7E057F0090DE
:1035B40000D3E08E048F05FF12712A900890E0FE7C
:1035C400A3E0FFEFC39DEE9C400FAC51AD52740FCE
:1035D400BC0004D39D50028002C232900089E0B442
:1035E4000227900892E0FEA3E0FF900890E0FCA37D
:1035F400E0FDEF2DFDEE3CFC74018C068D071200FE
:1036040039900890EEF0A3EFF0900890E0F8A3E072
:10361400900892C8F0A3C8F09000BBE06401600673
:10362400900891E0F55F8003755F00900085E0707D
:1036340006756F030232FC75BB18023CA8023CA855
:10364400900085E070030237B57E017F00E5BE126D
:10365400713AE5BD2FFF50010E8E598F5A9000CB61
:10366400E0B4010F7E0F7FFFAC59AD5A1271858E05
:10367400598F5A9000F0E0B40245AE59AF5A900009
:1036840024E0FCA3E0FDEDD39FEC9E400A900024CF
:10369400E559F0A3E55AF0AE59AF5A900026E0FC84
:1036A400A3E0FDEFD39DEE9C400A900026E559F07F
:1036B400A3E55AF0AE59AF5A74041200398F6190E1
:1036C40000F0E0704CAE59AF5A900024E0FCA3E047
:1036D400FDEFD39DEE9C40091271858E598F5A805F
:1036E40006755A00755900AE59AF5A741012713AE2
:1036F4009000EFE08E048F05FF12712A8C598D5AC9
:1037040074FFBC0009D39D4005855A61800375612F
:10371400FE9000BBE0B4010280030237B3A203B3FE
:10372400B3500E90008FE0A851B80005D3955250C5
:103734000280719000CCE08561F0A4FFAEF0746467
:103744008E048F05FF12712A8C598D5AE56B601611
:10375400E56BC394FE500F9000E5E0B402089000BE
:10376400D3E0640B60028017AE59AF5A74E712714C
:103774003AE56B8E048F05FF12712A8C598D5AAE6F
:1037840059AF5A900890E0FCA3E0FDEDD39FEC9E66
:103794004005855A5F800BA228B34006900891E04B
:1037A400F55F800BA228B34006900891E0F55F8096
:1037B40003756100900088E07006756F050232FCA5
:1037C40075BB19023CA8023CA8900088E070030273
:1037D400389CE55ED3955D400302389A900022E060
:1037E400FEA3E0FFE56512717D900022EEF0A3EFE9
:1037F400F09000F5E0B402247E017F00E5BE127172
:103804003AE5BD2FFF50010E8F048E057E0F7FFF1A
:10381400CDCCCD1271858E598F5A80147E017F00D4
:10382400E5BE12713AE5BD2FFF50010E8E598F5A35
:103834009000F5E07017AE59AF5A740A12713A74D9
:10384400518E048F05FF12712A8D658019AE59AF10
:103854005A740A12713A8F048E057E017F95CDCC7D
:10386400CD1270288F65E565D39464400375656453
:10387400900022E0FEA3E0FFE5652FFF50010E90CB
:103884000022EEF0A3EFF090008CE0048E048F058C
:10389400FF12712A8D6580037565329000D8E0703F
:1038A40006756F070232FC75BB13023CA8023CA8E4
:1038B4009000D8E0604A7E017F00E5BE12713AE5CF
:1038C400BD2FFF50010E8E598F5A74041200398F88
:1038D400669000DAE08566F0A4FDACF07464FF1233
:1038E400712A8D669000D9E08566F0A4FFAEF0746D
:1038F400FF8E048F05FF12712AED90006CF0800397
:10390400756600900086E07006756F090232FC75DA
:10391400BB17023CA8023CA8900086E0B4010280D8
:10392400030239B07E017F00E5BE12713AE5BD2F76
:10393400FF50010E8E598F5A9008E8E060199008E4
:10394400E8E014906B1A12008CE493FC740193FD6C
:10395400EDC39FEC9E400280069008E8E014F090CE
:1039640008E8E0C394B3501DAE59AF5A9008E8E09C
:1039740004906B1A12008CE493FC740193FDEFC362
:103984009DEE9C400280069008E8E004F09008E870
:10399400E0FE9000ACE08E0088F0A4FFAEF074640A
:1039A4008E048F05FF12712A8D678003756700905E
:1039B4000087E07006756F0B0232FC75BB16023C83
:1039C400A8023CA8900087E0B401028003023A5C9C
:1039D4007E017F00E5BE12713AE5BD2FFF50010E56
:1039E4008E598F5A9008E9E060199008E9E0149024
:1039F4006C8412008CE493FC740193FDEDC39FEC82
:103A04009E400280069008E9E014F09008E9E0C3C3
:103A140094B3501DAE59AF5A9008E9E004906C84F9
:103A240012008CE493FC740193FDEFC39DEE9C4063
:103A34000280069008E9E004F09008E9E0FE9000B6
:103A4400B2E08E0088F0A4FFAEF074648E048F059B
:103A5400FF12712A8D68800375680075BB1F023CD4
:103A6400A8023CA87E017F00E5BE12713AE5BD2F95
:103A7400FF50010E8E598F5A740912713A74E68EF2
:103A8400048F05FF12712A8D6A90008EE07006750E
:103A94006F0F0232FC75BB15023CA8023CA89000D3
:103AA4008EE07003023BF37E017F00E5BE12713AA3
:103AB400E5BD2FFF50010E8E598F5A740412003940
:103AC4008F6990008EE0B401159000E2E08569F002
:103AD400A4FFAEF07407120039EF9008E3F09000F1
:103AE4008EE0B402159000E2E08569F0A4FFAEF028
:103AF4007407120039EF9008E2F090008EE0B403EE
:103B0400028003023BD69000CFE07052E569C39473
:103B140019500FD2249000AEE09008E6F09008EB24
:103B2400E4F0E569D394644004A2244002802D901B
:103B340008EBE004F09008EBE0FE900121E0B5060C
:103B44000B9008E6E004F09008EBE4F09008E6E05F
:103B540064966006900121E07002C22480639000A4
:103B6400AEE070349000E2E08569F0A4FFAEF0743A
:103B7400FF8E048F05FF12712AED9008E6F0AE5116
:103B8400AF52741EBE0006D39F4002D224E561D317
:103B940094E54002C2248029E569C3940A500DAE1D
:103BA40051AF52741EBE0004D39F50028002D2242F
:103BB400E561D394E54002C2249000AEE09008E6AB
:103BC400F09008E6E0C39405500674059008E6F00A
:103BD400C22990008EE0B40414E569C3941950021C
:103BE400D229E569D394324002C229C224800375E4
:103BF40069009000E5E07006756F110232FC75BB38
:103C040014023CA8023CA89000E5E07003023C9535
:103C14007E017F00E5BE12713AE5BD2FFF50010E13
:103C24008E598F5A900125E075F010A4FDACF08CEC
:103C34005B8D5CEFD39DEE9C40091271858E598F8C
:103C44005A8006755A00755900AE59AF5A740E124F
:103C5400713A9000ECE08E048F05FF12712A8C5BA0
:103C64008D5C74FFBC00039D5005756BFF8003855C
:103C74005C6BE56B75F00BA4FFAEF09000D3E08EA7
:103C8400048F05FF12712A900894ECF0A3EDF080E4
:103C940003756B00900089E0600575BB1A8003759D
:043CA400BB188000C9
:103D0F000233050233080236410236440237CA0233
:103D1F0037CD0238B10238B402391902391C0239D1
:103D2F00C50239C8023A65023A68023A9F023AA2BE
:093D3F00023C08023C0B023CA806
:103CA800E56F75F00284AFF07E00EF4E7002D2EC43
:033CB800056F2273
:09716B002582F582500205832201
:0F008C0025E050020583258250020583F582226C
:10710900EF2F500205832582F582E5833E2EF58314
:017119002253
:10717D00CFC39FFF50011E22C3EF9DFFEE9CFE2249
:08718D000806B60002180622F4
:0D714800A3E004F07006127161E004F02273
:0E003900048007C3CE13CECF13CFD5E0F6223E
:10702800BC000FBE0008ED8FF084FFADF022E4FE37
:10703800FF22BE000DEF60FE54F0606F20E70302F0
:1070480070DEEAC0E0EBC0E078017A0075F001EE8E
:1070580020E710EF25E0FFEE33FE0AC5F023C5F068
:1070680030E7F0EA5407F9096A7A007B0060010802
:10707800C3EC9E40167004ED9F4010ED9FFDEC9E02
:10708800FCE5F0CA4ACA03F5F08005E5F003F5F01F
:10709800C3EE13FEEF13FFD9D77908CACBCAD8D0ED
:1070A800EAFEEBFFD0E0FBD0E0FA22EC8FF084FCA4
:1070B800ED54F045F0C48FF084FEEDC454F045F073
:1070C800C48FF084FDEEC4FE54F02DFFEE540F3C47
:1070D800FEADF07C0022790078008FF0EC7E08206D
:1070E800E70DC3CD33CD33C933C9C833C8DEF08407
:1070F80049F9E5F08FF0BE00E6FD7C00E9FFE8FE07
:017108002264
:0E713A00F88FF0A4FFE5F0CE88F0A42EFE2220
:10000300EF8DF0A4F9A8F0EF8CF0A428F8EE8DF0B2
:06001300A428FEE9FF2213
:10711A00600D782B027124007830D8FED5E0F82271
:10712A00EEC0E07E00127028EFFDEEFCD0E0FE22F9
:0C715500EEC0E07E00127028D0E0FE22A8
:03001B0002001EC2
:0300530002005652
:03009B00020071EF
:0300000002717416
:0971740075817575D000024C56BE
:0B004800E5822FF582E5833EF5832260
:0A7161000582D582021583158222F3
:10001E00C0E0C0F0C083C082C0D075D000124B5972
:0B002E00D0D0D082D083D0F0D0E032E0
:10005600C0E0C0F0C083C082C0D075D000124B5C37
:10006600D0D0D082D083D0F0D0E032C0E0C0F0C093
:1000760083C082C0D075D000124BBAD0D0D082D007
:0600860083D0F0D0E0324F
:00000001FF
